:020000040000FA
:040000007CEF4BF056
:080008005CEF00F000000000B5
:100010000000000000000000E8CF05F0D8CF06F097
:10002000E0CF07F00001E9CF0DF0EACF08F0E1CF13
:1000300009F0E2CF0AF0D9CF0BF0DACF0CF0F3CF12
:1000400014F0F4CF15F0FACF16F0FBCF17F000C084
:100050000FF001C010F002C011F003C012F004C094
:1000600013F09DAA37EF00F09EBA10EF0EF00FC00C
:1000700000F010C001F011C002F012C003F013C074
:1000800004F00DC0E9FF08C0EAFF09C0E1FF0AC0A3
:10009000E2FF0BC0D9FF0CC0DAFF14C0F3FF15C09C
:1000A000F4FF16C0FAFF17C0FBFF05C0E8FF07C04A
:1000B000E0FF06C0D8FF10000001E9CF1EF0EACF34
:1000C00019F0E1CF1AF0E2CF1BF0D9CF1CF0DACF54
:1000D0001DF0F3CF25F0F4CF26F0FACF27F0FBCFB9
:1000E00028F000C020F001C021F002C022F003C0BF
:1000F00023F004C024F0F2AA81EF00F0F2B4ABEFD9
:100100000DF020C000F021C001F022C002F023C099
:1001100003F024C004F01EC0E9FF19C0EAFF1AC0B2
:10012000E1FF1BC0E2FF1CC0D9FF1DC0DAFF25C0E4
:10013000F3FF26C0F4FF27C0FAFF28C0FBFF110021
:10014000F2CF0EF0F29CF29EF76A640FF66E010E8B
:10015000F722000EF86E0900F5500EBCF28C0EBEB0
:10016000F28E12000A0D436865636B696E67204169
:10017000637469766520454550524F4D20666F7215
:1001800020696E76616C696420446174610A0D00B7
:10019000F2CF0EF0F29CF29EF76AB40FF66E010EEB
:1001A000F722000EF86E0900F5500EBCF28C0EBE60
:1001B000F28E12002020436865636B696E672045EC
:1001C0004550524F4D207265636F72642030782520
:1001D0004C580A0D0000F2CF0EF0F29CF29EF76A26
:1001E000FA0FF66E010EF722000EF86E0900F550B8
:1001F0000EBCF28C0EBEF28E120044617461427924
:10020000746520584F5220436865636B427974656A
:10021000203D2025750D0A00F2CF0EF0F29CF29ED3
:10022000F76A3C0FF66E020EF722000EF86E090018
:10023000F5500EBCF28C0EBEF28E120009526573A0
:10024000746F72696E672066726F6D204261636BB6
:100250007570207265636F7264203078254C580A7F
:100260000D00F2CF0EF0F29CF29EF76A860FF66E4A
:10027000020EF722000EF86E0900F5500EBCF28C4B
:100280000EBEF28E12000909556E61626C65207413
:100290006F2066696E642076616C696420626163B8
:1002A0006B7570207265636F72640A0A0D00F2CF7D
:1002B0000EF0F29CF29EF76AD20FF66E020EF72253
:1002C000000EF86E0900F5500EBCF28C0EBEF28ED8
:1002D000120043616C6962726174696F6E206973A8
:1002E000204E4F542076616C6964210D0A0A00008B
:1002F000F2CF0EF0F29CF29EF76A140FF66E030E28
:10030000F722000EF86E0900F5500EBCF28C0EBEFE
:10031000F28E1200416C6C2063616C6962726174D0
:10032000696F6E20646174612069732076616C6905
:10033000640D0A00F2CF0EF0F29CF29EF76A580F9D
:10034000F66E030EF722000EF86E0900F5500EBC93
:10035000F28C0EBEF28E12000A0D55706461746943
:100360006E672063616C2064617461206261636BFD
:10037000757020636F706965730A0D00F2CF0EF01F
:10038000F29CF29EF76AA00FF66E030EF722000EA3
:10039000F86E0900F5500EBCF28C0EBEF28E120003
:1003A0002020436F6D706172696E67206261636BBC
:1003B000757020746F2076616C69642045455052D9
:1003C0004F4D2061646472657373203078254C58FA
:1003D0000A0D0000F2CF0EF0F29CF29EF76AF80FC1
:1003E000F66E030EF722000EF86E0900F5500EBCF3
:1003F000F28C0EBEF28E12005570646174696E67E5
:10040000206261636B7570207265636F7264203067
:1004100078254C580A0D0000F2CF0EF0F29CF29EA7
:10042000F76A3C0FF66E040EF722000EF86E090014
:10043000F5500EBCF28C0EBEF28E1200444F4E45AB
:100440000A0D0000F2CF0EF0F29CF29EF76A680FE0
:10045000F66E040EF722000EF86E0900F5500EBC81
:10046000F28C0EBEF28E12004154343544422046C6
:100470006F756E640A0D0000F2CF0EF0F29CF29ED2
:10048000F76A9C0FF66E040EF722000EF86E090054
:10049000F5500EBCF28C0EBEF28E1200466C6173EB
:1004A000682063686970206E6565647320746F20CE
:1004B00062652072657365740A0D506C65617365C1
:1004C000204379636C6520506F77657220616E649C
:1004D0002054727920416761696E0A0D0000F2CFE5
:1004E0000EF0F29CF29EF76A020FF66E050EF722EE
:1004F000000EF86E0900F5500EBCF28C0EBEF28EA6
:100500001200415432394320466F756E640A0D0063
:10051000F2CF0EF0F29CF29EF76A340FF66E050EE3
:10052000F722000EF86E0900F5500EBCF28C0EBEDC
:10053000F28E12000A0D4F6666736574203D202509
:10054000750A0D00F2CF0EF0F29CF29EF76A680F6A
:10055000F66E050EF722000EF86E0900F5500EBC7F
:10056000F28C0EBEF28E120057726974696E6700CB
:10057000F2CF0EF0F29CF29EF76A940FF66E050E23
:10058000F722000EF86E0900F5500EBCF28C0EBE7C
:10059000F28E12000A0D52656164696E6700F2CF37
:1005A0000EF0F29CF29EF76AC20FF66E050EF7226D
:1005B000000EF86E0900F5500EBCF28C0EBEF28EE5
:1005C00012005265616420257820696E737465613C
:1005D00064206F6620257820617420256C752028A2
:1005E0003078256C78290A0D0000F2CF0EF0F29CCD
:1005F000F29EF76A0E0FF66E060EF722000EF86EE8
:100600000900F5500EBCF28C0EBEF28E12000A0DDF
:10061000466C617368205465737420436F6D706C11
:10062000657465207769746820256C752062616443
:100630002062797465730A0D0000F2CF0EF0F29C0F
:10064000F29EF76A5E0FF66E060EF722000EF86E47
:100650000900F5500EBCF28C0EBEF28E120046411F
:10066000494C45440A0D54686520666C61736820E6
:100670006D656D6F72792069732064616D61676566
:10068000640A0D00F2CF0EF0F29CF29EF76AA80FFA
:10069000F66E060EF722000EF86E0900F5500EBC3D
:1006A000F28C0EBEF28E12004F4B0A0D0000F2CFFC
:1006B0000EF0F29CF29EF76AD20FF66E060EF7224B
:1006C000000EF86E0900F5500EBCF28C0EBEF28ED4
:1006D00012000A0A0D2050616765202575200A0A5C
:1006E0000D00F2CF0EF0F29CF29EF76A060FF66E46
:1006F000070EF722000EF86E0900F5500EBCF28CC2
:100700000EBEF28E12000A0D202025303275203ADE
:100710000000F2CF0EF0F29CF29EF76A360FF66EF2
:10072000070EF722000EF86E0900F5500EBCF28C91
:100730000EBEF28E120041542B42545343414E00E0
:10074000F2CF0EF0F29CF29EF76A640FF66E070E7F
:10075000F722000EF86E0900F5500EBCF28C0EBEAA
:10076000F28E120061746F0D0000F2CF0EF0F29C59
:10077000F29EF76A8E0FF66E070EF722000EF86EE5
:100780000900F5500EBCF28C0EBEF28E12004154E0
:100790002B42544E414D453D224D444C332D253086
:1007A000346C75220000F2CF0EF0F29CF29EF76AD4
:1007B000CA0FF66E070EF722000EF86E0900F5500C
:1007C0000EBCF28C0EBEF28E120041542B554152DB
:1007D00054434F4E4649472C0000F2CF0EF0F29C96
:1007E000F29EF76AFE0FF66E070EF722000EF86E05
:1007F0000900F5500EBCF28C0EBEF28E12003131A3
:10080000353230300000F2CF0EF0F29CF29EF76AE3
:100810002A0FF66E080EF722000EF86E0900F5504A
:100820000EBCF28C0EBEF28E120035373630300020
:10083000F2CF0EF0F29CF29EF76A540FF66E080E9D
:10084000F722000EF86E0900F5500EBCF28C0EBEB9
:10085000F28E1200313932303000F2CF0EF0F29CBD
:10086000F29EF76A7E0FF66E080EF722000EF86E03
:100870000900F5500EBCF28C0EBEF28E1200393615
:1008800030300000F2CF0EF0F29CF29EF76AA80F13
:10089000F66E080EF722000EF86E0900F5500EBC39
:1008A000F28C0EBEF28E12002C4E2C312C31000038
:1008B000F2CF0EF0F29CF29EF76AD40FF66E080E9D
:1008C000F722000EF86E0900F5500EBCF28C0EBE39
:1008D000F28E120041545A0D0000F2CF0EF0F29C3D
:1008E000F29EFC0FF66E080EF722000EF86E09005D
:1008F000F5500EBCF28C0EBEF28E12000200040007
:1009000007000A000E00110016001A001F00250043
:100910002A00310037003E0045004D0055005D00C3
:1009200066006F00790083008D009800A300AE0080
:10093000BA00C600D300E000ED00FB000901180179
:1009400027013601460156016601770188019A01A7
:10095000AC01BE01D101E401F7010B022002340217
:1009600049025F0274028A02A102B802CF02E702C2
:10097000FF0217033003490363037D039703B203A8
:10098000CD03E903050421043D045B0478049604C7
:10099000B404D204F1041105300550057105920527
:1009A000B305D505F70519063C065F068206A606BF
:1009B000CA06EF0614073A075F078607AC07D30796
:1009C000FA0722084A0873089C08C508EE081809A7
:1009D00043096E099909C409F0091C0A490A760AF3
:1009E000A40AD10A000B2E0B5D0B8C0BBC0BEC0B7D
:1009F0001D0C4E0C7F0CB00CE20C150D480D7B0D40
:100A0000AE0DE20D170E4B0E800EB60EEC0E220F41
:100A1000580F8F0FC70FFE0F37106F10A810E1107F
:100A20001B1155118F11CA11051241127D12B912F5
:100A3000F61233137013AE13EC132B146A14A914AB
:100A4000E91429156A15AB15EC152E167016B21699
:100A5000F51638177C17C017041849188E18D318C4
:100A600019195F19F2CF0EF0F29CF29EF76A880F07
:100A7000F66E0A0EF722000EF86E0900F5500EBC55
:100A8000F28C0EBEF28E1200507731313A6D702525
:100A9000346C646D7425356C756E7025356C7565B8
:100AA0006F6D0D0A0000F2CF0EF0F29CF29EF76A15
:100AB000CA0FF66E0A0EF722000EF86E0900F55006
:100AC0000EBCF28C0EBEF28E1200507731323A001C
:100AD000F2CF0EF0F29CF29EF76AF40FF66E0A0E59
:100AE000F722000EF86E0900F5500EBCF28C0EBE17
:100AF000F28E1200656F6D0D0A00F2CF0EF0F29CBF
:100B0000F29EF76A1E0FF66E0B0EF722000EF86EBD
:100B10000900F5500EBCF28C0EBEF28E120050771A
:100B200030310000F2CF0EF0F29CF29EF76A480FCF
:100B3000F66E0B0EF722000EF86E0900F5500EBC93
:100B4000F28C0EBEF28E1200694D444C332D2530CE
:100B5000346C75200000F2CF0EF0F29CF29EF76A22
:100B60007A0FF66E0B0EF722000EF86E0900F550A4
:100B70000EBCF28C0EBEF28E120076322E300000C9
:100B8000F2CF0EF0F29CF29EF76AA40FF66E0B0EF7
:100B9000F722000EF86E0900F5500EBCF28C0EBE66
:100BA000F28E1200507730350000F2CF0EF0F29C3A
:100BB000F29EF76ACE0FF66E0B0EF722000EF86E5D
:100BC0000900F5500EBCF28C0EBEF28E1200496E7A
:100BD00076616C696420496E7075740A0D00F2CFFD
:100BE0000EF0F29CF29EF76A020FF66E0C0EF722E0
:100BF000000EF86E0900F5500EBCF28C0EBEF28E9F
:100C000012002D2D3E3E0000F2CF0EF0F29CF29E1F
:100C1000F76A2C0FF66E0C0EF722000EF86E090024
:100C2000F5500EBCF28C0EBEF28E12004669726D4B
:100C300077617265202573574C0A0D00F2CF0EF0D4
:100C4000F29CF29EF76A600FF66E0C0EF722000E11
:100C5000F86E0900F5500EBCF28C0EBEF28E12003A
:100C60000A0D0A537769746368696E6720746F2090
:100C70004E6F726D616C204F7065726174696F6E3A
:100C80000A0D0000F2CF0EF0F29CF29EF76AA80F58
:100C9000F66E0C0EF722000EF86E0900F5500EBC31
:100CA000F28C0EBEF28E12000A0D54657374696EDA
:100CB0006720466C617368206D656D6F72790A0DEF
:100CC0000000F2CF0EF0F29CF29EF76AE60FF66E8D
:100CD0000C0EF722000EF86E0900F5500EBCF28CD7
:100CE0000EBEF28E12000A0D54657374696E672091
:100CF000416E616C6F672F4469676974616C204352
:100D00006F6E7665727465727300F2CF0EF0F29CAE
:100D1000F29EF76A2E0FF66E0D0EF722000EF86E99
:100D20000900F5500EBCF28C0EBEF28E1200546813
:100D30006973206369726375697420626F6172649C
:100D4000206E6565647320746F2062652072657023
:100D50006C616365642E0A0D0000F2CF0EF0F29C08
:100D6000F29EF76A7E0FF66E0D0EF722000EF86EF9
:100D70000900F5500EBCF28C0EBEF28E12000A0D68
:100D80005365742043616C6962726174696F6E208F
:100D9000446174650A0D0000F2CF0EF0F29CF29EE1
:100DA000F76ABC0FF66E0D0EF722000EF86E090002
:100DB000F5500EBCF28C0EBEF28E12000A0D536579
:100DC000742050726F62652053657269616C204EA9
:100DD000756D6265720A0D00F2CF0EF0F29CF29E04
:100DE000F76AFC0FF66E0D0EF722000EF86E090082
:100DF000F5500EBCF28C0EBEF28E12000A0D43614D
:100E00006C6962726174696F6E20436F6D706C659E
:100E100074650A0D0000F2CF0EF0F29CF29EF76AA4
:100E20003A0FF66E0E0EF722000EF86E0900F5501E
:100E30000EBCF28C0EBEF28E12002043616C696211
:100E4000726174696F6E2053756D6D617279200ADD
:100E50000D00F2CF0EF0F29CF29EF76A760FF66E5E
:100E60000E0EF722000EF86E0900F5500EBCF28C43
:100E70000EBEF28E120050726F6265204E616D657B
:100E8000203D204D444C332D2530346C750A0D0027
:100E9000F2CF0EF0F29CF29EF76AB40FF66E0E0ED1
:100EA000F722000EF86E0900F5500EBCF28C0EBE53
:100EB000F28E1200505349204F6666736574203DD0
:100EC00020256C750A0D0000F2CF0EF0F29CF29E08
:100ED000F76AEC0FF66E0E0EF722000EF86E0900A0
:100EE000F5500EBCF28C0EBEF28E1200505349200B
:100EF0005363616C6520203D20256C750A0D000050
:100F0000F2CF0EF0F29CF29EF76A240FF66E0F0EEF
:100F1000F722000EF86E0900F5500EBCF28C0EBEE2
:100F2000F28E12004952204F666673657420203D90
:100F300020256C640A0D0000F2CF0EF0F29CF29EA8
:100F4000F76A5C0FF66E0F0EF722000EF86E0900BE
:100F5000F5500EBCF28C0EBEF28E12004952205398
:100F600063616C653D20256C750A0D00F2CF0EF0B3
:100F7000F29CF29EF76A900FF66E0F0EF722000EAB
:100F8000F86E0900F5500EBCF28C0EBEF28E120007
:100F900043616C204461746520286D6D6464292070
:100FA0003D2025730A0D0000F2CF0EF0F29CF29E58
:100FB000F76ACC0FF66E0F0EF722000EF86E0900DE
:100FC000F5500EBCF28C0EBEF28E12002121205381
:100FD000617665207468697320496E666F726D6111
:100FE00074696F6E2021210A0D00F2CF0EF0F29C81
:100FF000F29EF76A0E0FF66E100EF722000EF86ED4
:101000000900F5500EBCF28C0EBEF28E12004C6937
:101010006E6520757020746865206C6173657273ED
:10102000206F6E2074686520256C754620686561A8
:101030007465720A0D00F2CF0EF0F29CF29EF76A10
:101040005A0FF66E100EF722000EF86E0900F550DA
:101050000EBCF28C0EBEF28E1200507265737320BD
:1010600074686520627574746F6E20756E74696C37
:10107000206C61736572732073746F7020666C618D
:101080007368696E6700F2CF0EF0F29CF29EF76A09
:10109000AA0FF66E100EF722000EF86E0900F5503A
:1010A0000EBCF28C0EBEF28E1200446F6E650A0DFD
:1010B0000000F2CF0EF0F29CF29EF76AD60FF66EA9
:1010C000100EF722000EF86E0900F5500EBCF28CDF
:1010D0000EBEF28E12009001B801F4011C02F2CF94
:1010E0000EF0F29CF29EF76A020FF66E110EF722D6
:1010F000000EF86E0900F5500EBCF28C0EBEF28E9A
:1011000012000A0D54657374204952205079726F91
:101110006D657465722043616C6962726174696F98
:101120006E2041636375726163790A0D0000F2CF2E
:101130000EF0F29CF29EF76A520FF66E110EF72235
:10114000000EF86E0900F5500EBCF28C0EBEF28E49
:1011500012004D6561737572656420256C754620BB
:1011600069732077697468696E20354620737065ED
:10117000630A0A0D0000F2CF0EF0F29CF29EF76AAD
:101180009A0FF66E110EF722000EF86E0900F55058
:101190000EBCF28C0EBEF28E1200495220547261C7
:1011A0006E7364756365722043616C696272617409
:1011B000696F6E20436F6D706C6574650A0A0D006F
:1011C000F2CF0EF0F29CF29EF76AE40FF66E110E6B
:1011D000F722000EF86E0900F5500EBCF28C0EBE20
:1011E000F28E12004D6561737572656420256C7511
:1011F00046204973204E6F742057697468696E20C9
:10120000537065632C2052652D43616C6962726175
:1012100074650A0A0D00F2CF0EF0F29CF29EF76A96
:101220003A0FF66E120EF722000EF86E0900F55016
:101230000EBCF28C0EBEF28E120043616C696272BB
:10124000617465204952205370616E0A0A0D0000D6
:10125000F2CF0EF0F29CF29EF76A740FF66E120E49
:10126000F722000EF86E0900F5500EBCF28C0EBE8F
:10127000F28E120043616C6962726174652049529A
:10128000206F66667365740A0D00F2CF0EF0F29C53
:10129000F29EF76AAE0FF66E120EF722000EF86E8F
:1012A0000900F5500EBCF28C0EBEF28E12004144C5
:1012B0005F75563D202530366C752054435F75565A
:1012C0003D202530356C7520446567463D2025302E
:1012D000336C750D0000F2CF0EF0F29CF29EF76AAF
:1012E000FA0FF66E120EF722000EF86E0900F55096
:1012F0000EBCF28C0EBEF28E12000A0D4952205323
:1013000063616C65203D20256C75203A2000F2CF8A
:101310000EF0F29CF29EF76A320FF66E130EF72271
:10132000000EF86E0900F5500EBCF28C0EBEF28E67
:1013300012000A0D4952204F6666736574203D20E5
:10134000256C64203A200000F2CF0EF0F29CF29E51
:10135000F76A6C0FF66E130EF722000EF86E090096
:10136000F5500EBCF28C0EBEF28E12005365742046
:101370004879647261756C69632050726573737526
:10138000726520746F20256C7550534920616E641E
:101390002050726573732074686520427574746F91
:1013A0006E00F2CF0EF0F29CF29EF76AC60FF66E58
:1013B000130EF722000EF86E0900F5500EBCF28CE9
:1013C0000EBEF28E12003200FA00EE02DC05F2CF01
:1013D0000EF0F29CF29EF76AF20FF66E130EF722F1
:1013E000000EF86E0900F5500EBCF28C0EBEF28EA7
:1013F00012005465737420507265737375726520A2
:101400005472616E7364756365722043616C6962C6
:10141000726174696F6E2041636375726163790AEA
:101420000D00F2CF0EF0F29CF29EF76A460FF66EB8
:10143000140EF722000EF86E0900F5500EBCF28C67
:101440000EBEF28E12004D656173757265642025C3
:101450006C75205053492069732077697468696EF0
:1014600020737065630A0A0D0000F2CF0EF0F29C43
:10147000F29EF76A8E0FF66E140EF722000EF86ECB
:101480000900F5500EBCF28C0EBEF28E12005072A6
:10149000657373757265205472616E7364756365EC
:1014A000722043616C6962726174696F6E20436F70
:1014B0006D706C6574650A0A0D00F2CF0EF0F29C37
:1014C000F29EF76ADE0FF66E140EF722000EF86E2B
:1014D0000900F5500EBCF28C0EBEF28E12004D6566
:1014E00061737572656420256C75205053492069BD
:1014F00073204E6F742057697468696E205370654D
:10150000632C2052652D43616C6962726174650AB7
:101510000A0D0000F2CF0EF0F29CF29EF76A380F2F
:10152000F66E150EF722000EF86E0900F5500EBC8F
:10153000F28C0EBEF28E120043616C6962726174AD
:1015400065205072657373757265205472616E7395
:101550006475636572205370616E0A0D0000F2CFEE
:101560000EF0F29CF29EF76A820FF66E150EF722CD
:10157000000EF86E0900F5500EBCF28C0EBEF28E15
:10158000120043616C696272617465205072657308
:1015900073757265205472616E7364756365722031
:1015A0004F66667365740A0D0000F2CF0EF0F29C70
:1015B000F29EF76ACE0FF66E150EF722000EF86E49
:1015C0000900F5500EBCF28C0EBEF28E1200507265
:1015D000657373757265205472616E7364756365AB
:1015E00072204F666673657420697320256C7520C0
:1015F0004D696C6C69766F6C74730A0D0000F2CFE4
:101600000EF0F29CF29EF76A220FF66E160EF7228B
:10161000000EF86E0900F5500EBCF28C0EBEF28E74
:1016200012005072657373757265205472616E7327
:101630006475636572204F666673657420697320F4
:101640004F5554204F4620544F4C4552414E434530
:101650000A0D0000F2CF0EF0F29CF29EF76A780FAE
:10166000F66E160EF722000EF86E0900F5500EBC4D
:10167000F28C0EBEF28E1200506C656173652061B3
:1016800074746163682061206E6577207472616E86
:1016900073647563657220616E6420747279206171
:1016A0006761696E0A0A0D00F2CF0EF0F29CF29E9D
:1016B000F76ACC0FF66E160EF722000EF86E0900D0
:1016C000F5500EBCF28C0EBEF28E12005053492023
:1016D0003D202530346C642009205053495F6D56FD
:1016E000203D202530346C640D00F2CF0EF0F29CCA
:1016F000F29EF76A0E0FF66E170EF722000EF86EC6
:101700000900F5500EBCF28C0EBEF28E12000A0DCE
:10171000505349204F6666736574203D20256C75D3
:10172000203A2000F2CF0EF0F29CF29EF76A480FAA
:10173000F66E170EF722000EF86E0900F5500EBC7B
:10174000F28C0EBEF28E12000A0D505349205363E4
:10175000616C65203D20256C75203A200000F2CF99
:101760000EF0F29CF29EF76A820FF66E170EF722C9
:10177000000EF86E0900F5500EBCF28C0EBEF28E13
:1017800012004A584E5F446567433D202530356C52
:101790006454435F4144616363756D3D2025303976
:1017A0006C750D00F2CF0EF0F29CF29EF76AC80F36
:1017B000F66E170EF722000EF86E0900F5500EBCFB
:1017C000F28C0EBEF28E12005261697365204A5887
:1017D0004E2074656D7020746F2061726F756E6439
:1017E0002035354320616E6420707265737320610B
:1017F000206B65790000F2CF0EF0F29CF29EF76A42
:101800001A0FF66E180EF722000EF86E0900F5504A
:101810000EBCF28C0EBEF28E12004A584E5F44652A
:1018200067433D202530356C640D0000F2CF0EF08B
:10183000F29CF29EF76A500FF66E180EF722000E19
:10184000F86E0900F5500EBCF28C0EBEF28E12003E
:101850004A584E5F5370616E3D202530346C7520C0
:1018600075565F5370616E3D202530366C752020B3
:10187000434A463D202530396C750D00F2CF0EF0FD
:10188000F29CF29EF76AA00FF66E180EF722000E79
:10189000F86E0900F5500EBCF28C0EBEF28E1200EE
:1018A00054435F414443282530337529203D20258A
:1018B00030356C55206D5620205053495F414443CC
:1018C000282530337529203D202530356C55206D75
:1018D00056200D00F2CF0EF0F29CF29EF76AF80F40
:1018E000F66E180EF722000EF86E0900F5500EBCC9
:1018F000F28C0EBEF28E120054454D505F414443AF
:10190000203D202530356C55206D560A0D50534929
:101910005F414443203D202530356C55206D560AEB
:101920000D00F2CF0EF0F29CF29EF76A460FF66EB3
:10193000190EF722000EF86E0900F5500EBCF28C5D
:101940000EBEF28E12004641494C45440A0D00007D
:10195000F2CF0EF0F29CF29EF76A740FF66E190E3B
:10196000F722000EF86E0900F5500EBCF28C0EBE88
:10197000F28E12000A0D20426C696E6B696E672050
:101980004C61736572732E202050726573732061F1
:10199000206B657920746F20717569742E200A0D93
:1019A0000000F2CF0EF0F29CF29EF76AC60FF66EC0
:1019B000190EF722000EF86E0900F5500EBCF28CDD
:1019C0000EBEF28E1200416D6269656E7420436531
:1019D0006C736975732054656D706572617475728E
:1019E00065203D202530326C6443200D0000F2CF8D
:1019F0000EF0F29CF29EF76A120FF66E1A0EF722A4
:101A0000000EF86E0900F5500EBCF28C0EBEF28E80
:101A10001200474F4F440D00F2CF0EF0F29CF29EA1
:101A2000F76A3C0FF66E1A0EF722000EF86E0900E8
:101A3000F5500EBCF28C0EBEF28E12004352495489
:101A40004943414C20200D00F2CF0EF0F29CF29E53
:101A5000F76A6C0FF66E1A0EF722000EF86E090088
:101A6000F5500EBCF28C0EBEF28E12000A0D5365BC
:101A70007269616C204E756D6265722069732030E9
:101A8000203A2000F2CF0EF0F29CF29EF76AA80FE7
:101A9000F66E1A0EF722000EF86E0900F5500EBC15
:101AA000F28C0EBEF28E12000A0D43616C2044616E
:101AB000746520286D6D646429203D202573203ACB
:101AC0002000F2CF0EF0F29CF29EF76AE60FF66E5F
:101AD0001A0EF722000EF86E0900F5500EBCF28CBB
:101AE0000EBEF28E12002D2D44617465206E6F744F
:101AF000204D6F6469666965642D2D0A0D00F2CF73
:101B00000EF0F29CF29EF76A220FF66E1B0EF72281
:101B1000000EF86E0900F5500EBCF28C0EBEF28E6F
:101B200012000A0D0A444941474E4F53544943207D
:101B30004D4F444520504F57455255500A0D000017
:101B40000501932D03D0010E016E02D0000E016E2F
:101B50000001FBEF0DF00C0ED66E305202E1315257
:101B600004E03050D8B4310630063D5202E13E5216
:101B700004E03D50D8B43E063D0605019253D8A47A
:101B800092070401B85302E1B95304E0B851D8B444
:101B9000B907B807B553D8A4B507B653D8A4B60744
:101BA000B753D8A4B7070501EB53D8A4EB0704013A
:101BB0005A53D8A45A073752D8A437063852D8A453
:101BC00038063952D8A43906325202E1335204E0C1
:101BD0003250D8B43306320681B009D0343C03D039
:101BE000353C01D003D0342AD8B4352A02D0356A26
:101BF000346A0001A5D7015210E0305202E131529F
:101C000001E00BD0316A640E306E0501942BD8B41C
:101C1000952B962BD8B4972B0001F29481EF00F00E
:101C20009EAAFED7AECF40F404013684336A190E63
:101C3000326E36A201D001D13F5326E140510A084D
:101C40000DE1415302E1425308E03F0E4125E96EA8
:101C5000000E4221EA6EEF6A3682EFD040510D0845
:101C600001E1EBD03F0E4125E96E000E4221EA6E04
:101C700040C4EFFF412BD8B4422B4251030802E28B
:101C8000426B416BDAD0D9D03F2D6CD040510D085A
:101C900011E13F0E4125E96E000E4221EA6EEF6A26
:101CA00036820A0E9EA8FED7AD6E0D0E9EA8FED7F8
:101CB000AD6EC3D04051080815E1415302E14253D3
:101CC00011E04151D8B442074107080E9EA8FED743
:101CD000AD6E200E9EA8FED7AD6E080E9EA8FED754
:101CE000AD6EABD042533DE13C50415D3AE24051D4
:101CF00060081BE240517A0818E3200E405F42C49E
:101D000003F04151412BD8B4422B0701076F3F0E1E
:101D10000725E96E000E0320EA6E40C4EFFF0401C0
:101D200040519EA8FED7AD6E88D040511F0819E2E1
:101D30004051600816E342C403F04151412BD8B42E
:101D4000422B0701076F3F0E0725E96E000E0320A7
:101D5000EA6E40C4EFFF040140519EA8FED7AD6E6D
:101D60006CD06BD03F510208D8A463D040510D080D
:101D700009E13F0E4125E96E000E4221EA6EEF6A4D
:101D800036825BD04051080815E1415302E14253CD
:101D900011E04151D8B442074107080E9EA8FED772
:101DA000AD6E200E9EA8FED7AD6E080E9EA8FED783
:101DB000AD6E43D042533CE13C50415D39E240516D
:101DC0002F0819E24051390816E342C403F041518B
:101DD000412BD8B4422B0701076F3F0E0725E96E50
:101DE000000E0320EA6E40C4EFFF040140519EA89C
:101DF000FED7AD6E22D040512D081AE1415318E1B3
:101E0000425316E142C403F04151412BD8B4422B56
:101E10000701076F3F0E0725E96E000E0320EA6EEB
:101E200040C4EFFF040140519EA8FED7AD6E05D01F
:101E300004D03F51030801E100D09E9A000137EF22
:101E400000F08790999087929992879699968798B3
:101E50009998879A999A878C999C879E999E809049
:101E60009290809292925CEF4EF0C70ED56E0C0E5F
:101E7000D66EF28A5EEF4EF00601DA513A5C01E16D
:101E800004D0DAC63AF03B6A396A0001000C040E4D
:101E9000026E016AEA6A3F0EE96EEE6A012EFDD714
:101EA000022EFBD7369436920401426B416B00013F
:101EB000000CF29E9E9AA49A9E98A498AB6AAB8E50
:101EC0009D8AAB88F28CAC6AAC8AAC84F28E6DEFE2
:101ED0000FF03E6A3D6ADBDFECD70601DB6BDBC649
:101EE0003FF4A26A9D8A3E6A320E3D6E0001000CEC
:101EF000D8C6AFFF6BEF4EF082869496829A949A82
:101F0000C79EC79C010EC66EC688C68A9E96000CE8
:101F1000200E016E050EEA6E5F0EE96EEE6A012E6E
:101F2000FDD7400E016E040EEA6EBE0EE96EEE6A3B
:101F3000012EFDD7200E016E050EEA6E0D0EE96E24
:101F4000EE6A012EFDD7200E016E050EEA6E360EEA
:101F5000E96EEE6A012EFDD705010A6B460E096F88
:101F6000906B640E8F6F010E0401B96F2C0EB86F69
:101F700000016FEF4EF0C69ABFEF0FF0FCD78296CC
:101F8000000000000000000000000000829000003F
:101F9000000000000000000000000601EB6BEB51A8
:101FA0000F0810E38286000000000000000000001F
:101FB0000000829600000000000000000000000009
:101FC000EB2BEDD782889498EB6BEB510F0810E365
:101FD00082860000000000000000000000008296E1
:101FE000000000000000000000000000EB2BEDD717
:101FF00082809488000000000000000000000000C3
:1020000082968290EB6BEB510F0810E38286000002
:1020100000000000000000000000829600000000A8
:102020000000000000000000EB2BEDD78298949890
:10203000EB6BEB510E0810E38286000000000000FD
:102040000000000000008296000000000000000078
:1020500000000000EB2BEDD78280948800014CDF5C
:10206000000C949082800401AB6BAD6BAC6BAF6BDA
:10207000AE6B0A0E016E040EEA6EA10EE96EEE6AF8
:10208000012EFDD700017ADF71EF4EF00601F65107
:10209000FC0F15E2040F000163EF10F0C698C79C17
:1020A00006010DD0C698C78C060109D0C688C79C0A
:1020B000060105D0C688C78C060101D00601C69A64
:1020C000C68A0001000CF2CF0EF0F29CF29EE824CA
:1020D000F70FF66E200EF76ED8B0F72A000EF86EE6
:1020E000FB6E0A00F550FA6E0800F5500EBCF28C3B
:1020F0000EBEF28EF96E9C20A420AC20B4209E96D9
:10210000F8C6C9FF9EA6FED7C9CF4DF4000C9E9617
:10211000C96A9EA6FED7C9CF01F0000C080E0601C1
:10212000F86F0001ECDFF3DF0150B0EF10F0100E9C
:102130000601F86F0001E3DFF6C6F8F6E0DFBEEF58
:1021400010F0180E0601F86F0001D9DFE0DF015032
:10215000BFEF10F0020E0601F66F000197DFDED729
:1021600001C0F5F60601F5513C0B0C0803E0FF0E2B
:10217000016E10D0060EF66F0001D9D7E2D701C06C
:10218000F5F60601F551060803E0FF0E016E02D0D8
:10219000000E016E0001000C060EEA6EEB0EE96EF9
:1021A000EF500FE0080E016E006A002EFED7012EE0
:1021B000FBD7190E006E002EFED700000000EF2E98
:1021C000F1D7000C020E0601F66F00015FDFFF0E73
:1021D0000601F86F000193DFFF0E0601F86F0001A2
:1021E0008EDFFF0E0601F86F000189DFFF0E06018A
:1021F000F86F000184DFFF0E0601F86F00017FDF3A
:10220000000C8284828094928292A4DF01BE01D06D
:1022100017D082828782320E0601EB6F0001BCDF8D
:102220008792320E0601EB6F0001B6DF8292CADFA1
:102230008282140E006E002EFED700008292E5D737
:10224000828273EF4EF082828280020E0601F66F68
:1022500000011CDF949482947DDF01BE01D017D071
:1022600082848782320E0601EB6F000195DF879230
:10227000320E0601EB6F00018FDF8294A3DF8284B0
:10228000140E006E002EFED700008294E5D78284E3
:1022900075EF4EF0D9C6B0F40401B051FB0F1EE249
:1022A000050F000170EF11F0040118D00C0E0601AB
:1022B000DA6F0001E1DD040111D00D0E0601DA6FC5
:1022C0000001DADD04010AD00E0E0601DA6F00010A
:1022D000D3DD040103D0040101D004010001000C8E
:1022E000F2CF0EF0F29CF29EE824110FF66E230E50
:1022F000F76ED8B0F72A000EF86EFB6E0A00F550A4
:10230000FA6E0800F5500EBCF28C0EBEF28EF96E1D
:10231000A822AC22BA22C822D6220601D96B00011B
:10232000B9DF0401B16B000E016E0001000C050164
:10233000956B946B976B966B996B986B000179EF2B
:102340004EF00601D951F60F3AE20A0F0001E3EF11
:1023500011F0080E0601DA6F00018EDD06012FD0A4
:10236000090E0601DA6F000187DD060128D00B0E89
:102370000601DA6F000180DD060121D006011FD0C1
:1023800006011DD0050E0601DA6F000175DD06019C
:1023900016D0020E0601DA6F00016EDD06010FD0C5
:1023A000060E0601DA6F000167DD060108D0010E96
:1023B0000601DA6F000160DD060101D00601D9C611
:1023C00093F50001000CF2CF0EF0F29CF29EE8248F
:1023D000F70FF66E230EF76ED8B0F72A000EF86EE0
:1023E000FB6E0A00F550FA6E0800F5500EBCF28C38
:1023F0000EBEF28EF96E8423AE23BC239223A0235B
:1024000080237C236E23602352230601E2810B0E7E
:10241000F86F000174DE7BDE01C0E1F60601E151D8
:10242000800B000A03E0FF0E016E33D03B0EF86F05
:10243000000165DE0601E16BE151020823E3020EB3
:10244000D880E155036A4D0F016E040E032201C0CE
:10245000E4F603C0E5F600015ADEE5C6EAFFE4C68D
:10246000E9FF01C0EFFF020ED8800601E155036AC3
:102470004D0FE96E040E0320EA6EEF52D8A4E291EC
:10248000E12BDAD7E2A103D0FE0E016E02D0000EDE
:10249000016E0001000C0701016B026B010E036F5E
:1024A000DA6AD96A060E066FF90E056F060EEA6E35
:1024B000FD0EE96E06C7E2FF05C7E1FF03C704F79B
:1024C000D890E550EE02F3500123F4500223042F7C
:1024D000F7D701C7DEFF02C701F7026BD8B0022BA6
:1024E000052BD8B4062B032B03510508DFE10001AF
:1024F000000C0601DC6BDD6BDE6BDF6B828282849D
:102500008280878E9D9A829200017FDF01C0E0F673
:1025100082829D8A879E0601E0BF6AD04FC40CF577
:102520004EC40BF505010B512E270C512F23000E25
:1025300030233123D8902D35036A0D0FE96E050E37
:102540000320EA6EECCF03F0ED52EF502E5F035004
:102550002F5B000E305B315BD8902D35036A0D0F79
:10256000E96E050E0320EA6E0CC5ECFFED520BC5BB
:10257000EFFF2D2B2D510F0801E22D6B313106019C
:10258000E56F050130310601E46F05012F310601C9
:10259000E36F05012E310601E26FE533E433E333E7
:1025A000E233E533E433E333E233E533E433E33377
:1025B000E2330F0EE517E5C6FCF6E4C6FBF6E3C60C
:1025C000FAF6E2C6F9F60701006B0601FF6B160E7C
:1025D000FE6FDA0EFD6F00015EDF02C0DCF603C0A5
:1025E000DDF60601DE6BDF6BDDC633F5DCC632F5EA
:1025F000878E9D9A020EF66F000148DD829405DFFA
:1026000001C0E0F682849D8A879E0601E0BF6AD001
:102610004FC435F54EC434F50501345157273551B3
:102620005823000E59235A23D8905635036A360F83
:10263000E96E050E0320EA6EECCF03F0ED52EF5089
:10264000575F0350585B000E595B5A5BD890563564
:10265000036A360FE96E050E0320EA6E35C5ECFFFE
:10266000ED5234C5EFFF562B56510F0801E2566B61
:102670005A310601E56F050159310601E46F050184
:1026800058310601E36F050157310601E26FE5336A
:10269000E433E333E233E533E433E333E233E53386
:1026A000E433E333E2330F0EE517E5C6FCF6E4C688
:1026B000FBF6E3C6FAF6E2C6F9F60701006B06017F
:1026C000FF6B160EFE6FDA0EFD6F0001E4DE02C036
:1026D000DCF603C0DDF60601DE6BDF6BDDC65CF504
:1026E000DCC65BF50001000C500E0601EA6FC30E5C
:1026F000EB6F8794EA51D8B4EB07EA07EA5306E197
:10270000EB5304E18784FF0E016E10D0D70EF86FF3
:102710000001F5DCFCDC0150800B000AD8A402D0DB
:102720000601E8D78784000E016E06010001000C47
:10273000010E0601F66F0001A9DC8794D70E060191
:10274000F86F0001DCDCE3DC01C0E2F687840601FF
:10275000E2513C0B2C0803E0000E016E02D0E2C6F1
:1027600001F00001B5EF13F0E3D70150010B0601B2
:10277000E16FE1C601F00001BFEF13F0F5D70152A0
:1027800003E0000E016E28D0AFDF015203E0FF0E20
:10279000016E22D0010E0601F66F000177DC8794EE
:1027A0003D0E0601F86F0001AADC2A0E0601F86F43
:1027B0000001A5DC800E0601F86F0001A0DCA60E6A
:1027C0000601F86F00019BDC87840A0E0601EB6F9F
:1027D0000001E2DC010E016E000C010E0601F66F35
:1027E000000154DC87949F0E0601F86F000187DC1E
:1027F0008EDC01C0DAF60601DA511F0804E0878496
:10280000FF0E016E10D0000182DC01C0DAF6060175
:10281000DA51E00B200804E08784FF0E016E03D03C
:102820008784000E016E000137EF14F099948784BD
:102830009698849896968496910E006E002EFED7F8
:1028400000008486140E0601EB6F0001A5DC040174
:10285000576B000149DF015203E0FF0E016E13D0F8
:102860008DDF01AE03D0FF0E016E0DD0B6D701BED5
:1028700001D003D0FF0E016E06D0010E0401576F88
:102880008488000E016E000126EF15F0956AAA0EED
:102890008C6E550E886E856E8492849400000000C4
:1028A000000000000000000084848C6E2A0E886EF8
:1028B000AA0E856E84940000000000000000000055
:1028C00000008484900E8C6E550E886E856E849404
:1028D00000000000000000000000000084848482EA
:1028E0000A0E0601EB6F000157DCBEEF14F0060183
:1028F000E46BFF0E956EE351886EE2C685FF84920D
:10290000849083CFE4F684808482E4C601F00001E1
:10291000000C956AAA0E8C6E550E886E856E849298
:102920008494000000000000000000000000848487
:102930008C6E2A0E886EAA0E856E849400000000AC
:1029400000000000000000008484F00E8C6E550E24
:10295000886E856E84940000000000000000000076
:102960000000848484820A0E0601EB6F000114DCEF
:10297000000C0601DC6BDD6B000188D70601E36B00
:10298000E26B0001B4DF01C0DCF60601DC511F0878
:1029900005E00001BEDFFF0E0601DD6FE36B010EF7
:1029A000E26F0001A4DF01C0DCF60601DC51DC08A7
:1029B0000AE00001AEDF0601DD5303E1FF0EDD6F2B
:1029C00002D0FD0EDD6F0001A4DF0601DDC601F0BF
:1029D000000101EF15F00601DA6B010EDB6F848256
:1029E00096928480969084849694856A976A886A81
:1029F0009A6A836AFF0E956EDB51050814E30001A5
:102A0000B8D701C0DAF60601DABF01D005D0DB2B5A
:102A10000401526B06D00601010E0401526F06013B
:102A200002D00601E9D7010E0401526F000E016EBB
:102A3000000129EF15F00601D86BD96B04019E6BDC
:102A40009D6B9C6B9B6B5A6B0001F0D601C0D8F656
:102A5000C2D701C0D9F60601D8AF06D0D9BF01D080
:102A600003D0FF0E016E02D0000E016E00019EEF3A
:102A70004AF00601EEBF10D00F0E006EED390016C1
:102A80000A0E005C03E2300E002602D0EE51002652
:102A900000509EA8FED7AD6E0F0EED170A0EED5D2D
:102AA00002E2300E02D0EE9FEE51ED27ED519EA8CE
:102AB000FED7AD6E0001000C0601E651016AE55D2E
:102AC00003E2E5C600F00CD0006A080EE76FE537B8
:102AD0000036E651005CD8B0006E0136E72FF7D71C
:102AE0000001000C0150E3C6E5F6640E0601E66F36
:102AF0000001E2DF00C0E3F60150300E08E10601FC
:102B0000E4A30ED0E4B70CD0E4B9200E04D0060143
:102B1000E497E499E481012601509EA8FED7AD6EAA
:102B2000E3C6E5F60A0EE66F0001C6DF00C0E3F675
:102B30000150300E08E10601E4B70BD0E4A109D042
:102B4000E4B9200E0001012601509EA8FED7AD6E0B
:102B50000601300EE327E3519EA8FED7AD6E0001BB
:102B6000000C010E0601E06FD9531FE0E16BE1514B
:102B70000001A0EC00F00601E12B006E00509EA8C1
:102B8000FED7AD6E290EE15DF2E1040EE26F2E0E6E
:102B90009EA8FED7AD6EE22FFAD70A0E9EA8FED7EA
:102BA000AD6E0D0E9EA8FED7AD6EDF6B400EDE6FD4
:102BB000DF53D8A430D1DE515508D8A02CD1D9513B
:102BC000010825E2E16BE1510001C8EC00F00601CB
:102BD000E12B006E00509EA8FED7AD6E1B0EE15D8E
:102BE000F2E1DFC6EDF6370EEE6F000142DFDEC622
:102BF000EDF6370E0601EE6F00013BDF0A0E9EA8D0
:102C0000FED7AD6E0D0E9EA8FED7AD6E0601F2CFBB
:102C1000E1F6F29CF29EDFC6AAFFDEC6A9FFA69CE3
:102C2000A69EA680A850E1BDF28CE1BFF28EDA6FBD
:102C3000160EDE25E16F000EDF21F2CFE3F6F29CE7
:102C4000F29EAA6EE1C6A9FFA69CA69EA680A850E9
:102C5000E3BDF28CE3BFF28EDB6FDA51DB19FF08C4
:102C600001E1D3D0D951010821E2DA51DB19E16F3A
:102C7000E26BE2510001EBEC00F00601E22B006E8A
:102C800000509EA8FED7AD6E190EE25DF2E1E1C6DE
:102C9000E3F61B0EE46F000125DF0D0E9EA8FED7A4
:102CA000AD6E0A0E9EA8FED7AD6E06012C0EDE2577
:102CB000DC6F000EDF21DD6FD951010825E2E16BE9
:102CC000E15100010CEC01F00601E12B006E005017
:102CD0009EA8FED7AD6E200EE15DF2E1DDC6EDF6F9
:102CE000370EEE6F0001C5DEDCC6EDF6370E0601CD
:102CF000EE6F0001BEDE0A0E9EA8FED7AD6E0D0E71
:102D00009EA8FED7AD6E0601F2CFE1F6F29CF29ED0
:102D1000DDC6AAFFDCC6A9FFA69CA69EA680A85079
:102D2000E1BDF28CE1BFF28EDA6F160EDC25E16FA9
:102D3000000EDD21F2CFE3F6F29CF29EAA6EE1C610
:102D4000A9FFA69CA69EA680A850E3BDF28CE3BF77
:102D5000F28EDB6FDA51DB19FF0838E1DFC6AAFF1C
:102D6000DEC6A9FFDAC6A8FFA69CA69EA684F2CF5F
:102D700000F0F29CF29E0F01550EA76EAA0EA76EF0
:102D8000A682A6B2FED7A6940050F212160E060135
:102D9000DE25E16F000EDF21E26FAA6EE1C6A9FF1A
:102DA000DBC6A8FFA69CA69EA684F2CF00F0F29CEC
:102DB000F29E0F01550EA76EAA0EA76EA682A6B2AE
:102DC000FED7A6940050F21221D006012C0EDC276B
:102DD000000EDD23DD51030816E2D95101080FE290
:102DE000E16BE151000131EC01F00601E12B006ED5
:102DF00000509EA8FED7AD6E270EE15DF2E1E06BBC
:102E00000F0104D00601040057D70F010601DE2B85
:102E1000D8B4DF2BCDD6E05314E1D9530FE0E16BEA
:102E2000E151000157EC01F00601E12B006E00506A
:102E30009EA8FED7AD6E1C0EE15DF2E1FF0E016EA5
:102E400013D0D9530FE0E16BE151000178EC01F0B0
:102E50000601E12B006E00509EA8FED7AD6E1F0E3E
:102E6000E15DF2E1000E016E0001000C0601D95394
:102E70001FE0E26BE25100019AEC01F00601E22B47
:102E8000006E00509EA8FED7AD6E210EE25DF2E10D
:102E9000040EE36F2E0E9EA8FED7AD6EE32FFAD779
:102EA0000A0E9EA8FED7AD6E0D0E9EA8FED7AD6E83
:102EB000E16B400EE06FE153D8A4FBD0E051550820
:102EC000D8A0F7D0D951010825E2E26BE251000108
:102ED000BEEC01F00601E22B006E00509EA8FED76A
:102EE000AD6E2D0EE25DF2E1E1C6EDF6370EEE6F4E
:102EF0000001BFDDE0C6EDF6370E0601EE6F000102
:102F0000B8DD0A0E9EA8FED7AD6E0D0E9EA8FED7A8
:102F1000AD6E0601F2CFE2F6F29CF29EE1C6AAFF88
:102F2000E0C6A9FFA69CA69EA680A850E2BDF28C92
:102F3000E2BFF28EDC6F160EE025E26F000EE1219B
:102F4000F2CFE4F6F29CF29EAA6EE2C6A9FFA69C1E
:102F5000A69EA680A850E4BDF28CE4BFF28EDD6F81
:102F6000DC51DD19FF0801E0A0D02C0EE025DE6F5A
:102F7000000EE121DF6FDF510308D8A096D0F2CF19
:102F8000E2F6F29CF29EDFC6AAFFDEC6A9FFA69C6F
:102F9000A69EA680A850E2BDF28CE2BFF28EDA6F48
:102FA000160EDE25E26F000EDF21F2CFE4F6F29C72
:102FB000F29EAA6EE2C6A9FFA69CA69EA680A85075
:102FC000E4BDF28CE4BFF28EDB6FDC51DA5D67E0CA
:102FD000D95101082DE2040EE26F200E9EA8FED703
:102FE000AD6EE22FFAD7E36BE3510001EAEC01F09A
:102FF0000601E32B006E00509EA8FED7AD6E190EA1
:10300000E35DF2E1DFC6EDF6370EEE6F000131DD74
:10301000DEC6EDF6370E0601EE6F00012ADD0A0E60
:103020009EA8FED7AD6E0D0E9EA8FED7AD6E060112
:10303000DFC6AAFFDEC6A9FFDCC6A8FFA69CA69E27
:10304000A684F2CF00F0F29CF29E0F01550EA76EFF
:10305000AA0EA76EA682A6B2FED7A6940050F212C0
:10306000160E0601DE25E26F000EDF21E36FAA6E69
:10307000E2C6A9FFDDC6A8FFA69CA69EA684F2CF45
:1030800000F0F29CF29E0F01550EA76EAA0EA76EDD
:10309000A682A6B2FED7A6940050F21206012C0E0C
:1030A000DE27000EDF23040066D7E02BD8B4E12B27
:1030B00002D7D9530FE0E26BE25100010CEC02F0B1
:1030C0000601E22B006E00509EA8FED7AD6E060EE4
:1030D000E25DF2E10001000CAA6A010EA96EDDC6F4
:1030E000A8FFA69CA69EA684F2CF00F0F29CF29EBA
:1030F0000F01550EA76EAA0EA76EA682A6B2FED726
:10310000A6940050F2120601DDC6DEF6DE1FAA6AA2
:10311000160EA96EDEC6A8FFA69CA69EA684F2CFB8
:1031200000F0F29CF29E0F01550EA76EAA0EA76E3C
:10313000A682A6B2FED7A6940050F2120001000C9F
:103140000601D86BD96BF2CFDAF6F29CF29EAA6A2E
:10315000010EA96EA69CA69EA680A850DABDF28C90
:10316000DABFF28ED86FF2CFDAF6F29CF29EAA6A3C
:10317000160EA96EA69CA69EA680A850DABDF28C5B
:10318000DABFF28ED96FD851D919FF0804E0DD6B90
:103190000001A2DF06010001DEEF18F00601D96B85
:1031A0000001DFDC01BE01D004D03696FF0E016EB7
:1031B00008D00601D96B000159DEC2D73686000E51
:1031C000016EB4EF4AF0385202E0938801D0819842
:1031D00037521BE136A015D0000E87B6010E010A4A
:1031E000016EE8B002D0879601D08786000E87B8BE
:1031F000010E010A016EE8B002D0879801D08788DD
:1032000002D087968798190E376E395201E0F1D1B6
:103210003A50F00FD8B0EDD1100FFAEF1AF03B5042
:10322000000A05E0010A09E0030A0DE012D08790C8
:103230008792640E396E3B2A12D087808782140EE3
:10324000396E3B2A0CD087908792140E396E3B2A38
:1032500006D087808782140E396E3B6A00D0C9D1B0
:103260003B50000A05E0010A09E0030A0DE012D014
:10327000879087820A0E396E3B2A12D087908792F8
:10328000140E396E3B2A0CD0879087820A0E396E55
:103290003B2A06D087908792320E396E3B6A00D067
:1032A000A8D13B50000A05E0010A09E0030A0DE03D
:1032B00012D0878087920A0E396E3B2A12D08790EF
:1032C0008792140E396E3B2A0CD0879087820A0EA3
:1032D000396E3B2A06D087908792320E396E3B6A50
:1032E00000D087D13B50000A05E0010A09E0030A3B
:1032F0000DE012D0878087920A0E396E3B2A12D0D9
:1033000087908792140E396E3B2A0CD08780879263
:103310000A0E396E3B2A06D087908792320E396E9C
:103320003B6A00D066D13B50000A09E0010A0DE07B
:10333000030A11E0010A15E0070A19E01ED0879080
:103340008792640E396E3B2A1ED087808782140EC6
:10335000396E3B2A18D087908792140E396E3B2A1B
:1033600012D087808782140E396E3B2A0CD087904A
:103370008792140E396E3B2A06D087808782140EFE
:10338000396E3B6A00D035D13B50000A09E0010A92
:103390000DE0030A11E0010A15E0070A19E01ED04A
:1033A000879087820A0E396E3B2A1ED087908792BB
:1033B000140E396E3B2A18D0879087820A0E396E18
:1033C0003B2A12D087908792140E396E3B2A0CD07C
:1033D000879087820A0E396E3B2A06D087908792A3
:1033E000320E396E3B6A00D004D13B50000A09E02E
:1033F000010A0DE0030A11E0010A15E0070A19E0CD
:103400001ED0878087920A0E396E3B2A1ED0879085
:103410008792140E396E3B2A18D0879087820A0E45
:10342000396E3B2A12D087908792140E396E3B2A50
:103430000CD0879087820A0E396E3B2A06D087907F
:103440008792320E396E3B6A00D0D3D03B50000ACF
:1034500009E0010A0DE0030A11E0010A15E0070A7C
:1034600019E01ED0878087920A0E396E3B2A1ED043
:1034700087908792140E396E3B2A18D087808792E6
:103480000A0E396E3B2A12D087908792140E396E3D
:103490003B2A0CD0879087820A0E396E3B2A06D0D1
:1034A00087908792320E396E3B6A00D0A2D03B5093
:1034B000000A09E0010A0DE0030A11E0010A15E023
:1034C000070A19E01ED0878087920A0E396E3B2AC0
:1034D0001ED087908792140E396E3B2A18D08780B1
:1034E00087920A0E396E3B2A12D087908792140E6B
:1034F000396E3B2A0CD0878087920A0E396E3B2AA0
:1035000006D087908792320E396E3B6A00D071D018
:103510003B50000A03E0010A07E00CD08790878245
:103520000A0E396E3B2A06D0879087920A0E396EB2
:103530003B6A00D05ED03B5206E0879087820A0E3D
:10354000396E3B6A06D0879087925A0E396E010E0B
:103550003B6E4FD03B5206E087908782320E396E29
:103560003B6A06D087908792320E396E010E3B6E11
:1035700040D03B50000A03E0010A07E00CD08780EE
:1035800087920A0E396E3B2A06D0879087920A0EE0
:10359000396E3B6A00D02DD03B5206E0878087927F
:1035A000050E396E3B6A06D0879087925F0E396EA2
:1035B000010E3B6E1ED03B5206E0878087920A0EBA
:1035C000396E3B6A06D0879087925A0E396E010E8B
:1035D0003B6E0FD03B5206E087808792320E396EE9
:1035E0003B6A06D087908792320E396E010E3B6E91
:1035F00000D0000CF2CF0EF0F29CF29EE824250FD2
:10360000F66E360EF76ED8B0F72A000EF86EFB6E27
:103610000A00F550FA6E0800F5500EBCF28C0EBE92
:10362000F28EF96E10353635543572359835B6351B
:10363000D4351E326032A232E43226338833EA3384
:103640004C34AE34E0C603F00601DFC6E9FFE0C645
:10365000EAFFEF504F0803E0000E016E11D0010E9B
:10366000DF25016E000EE021036E01C0E9FFEA6E66
:10367000EF504B0803E0000E016E02D0010E016E08
:103680000001A9EF1BF0E0C603F00601DFC6E9FF69
:10369000E0C6EAFFEF50450803E0000E016E3ED0A1
:1036A000010EDF25016E000EE021036E01C0E9FF6F
:1036B000EA6EEF50520803E0000E016E2FD0020EAA
:1036C000DF25016E000EE021036E01C0E9FFEA6E06
:1036D000EF50520803E0000E016E20D0030EDF25EC
:1036E000016E000EE021036E01C0E9FFEA6EEF50AB
:1036F0004F0803E0000E016E11D0040EDF25016EAD
:10370000000EE021036E01C0E9FFEA6EEF5052089F
:1037100003E0000E016E02D0010E016E0001000CEC
:1037200047EC0FF00D0E9EA8FED7AD6EDEC63EF044
:10373000DDC63DF00A0E386E3D5202E13E5220E0F9
:1037400042DD36A21CD00601E06B3F0EDF6F0001A8
:1037500079D7015205E047EC0FF0000E016E12D050
:103760000601E06B3F0EDF6F00018DDF015205E0C7
:1037700047EC0FF0FE0E016E05D047EC0FF0DCD7E2
:10378000FF0E016E000C610E9EA8FED7AD6E740E8A
:103790009EA8FED7AD6E0601DE6B0A0EDD6F00013E
:1037A000BFDF01BE03D0000E016E47D0610E9EA8A0
:1037B000FED7AD6E740E9EA8FED7AD6E0601DE6B11
:1037C0000A0EDD6F0001ACDF01BE03D0000E016EFA
:1037D00034D0030E0601D96F2B0E9EA8FED7AD6E16
:1037E000D92FFAD7C80EEB6F0001CCEC10F0610EA8
:1037F0009EA8FED7AD6E740E9EA8FED7AD6E0601D4
:10380000DE6B0A0EDD6F00018BDF01BE14D00601F6
:10381000D96BD9510001A0EC03F00601D92B006E41
:1038200000509EA8FED7AD6E040ED95DF2E1010EE8
:10383000016E000102D0FF0E016EA5EF1DF0060122
:10384000DD6BDD510001D3EC03F00601DD2B006ED2
:1038500000509EA8FED7AD6E0E0EDD5DF2E1D9518F
:103860000D0A000105E0170A14E04A0A23E033D0EC
:103870000601DD6BDD510001EDEC03F00601DD2BEF
:10388000006E00509EA8FED7AD6E060EDD5DF2E123
:1038900033D00601DD6BDD51000103EC04F00601BD
:1038A000DD2B006E00509EA8FED7AD6E050EDD5DCF
:1038B000F2E122D00601DD6BDD51000118EC04F0CD
:1038C0000601DD2B006E00509EA8FED7AD6E050EE2
:1038D000DD5DF2E111D00601DD6BDD5100012DEC63
:1038E00004F00601DD2B006E00509EA8FED7AD6EE1
:1038F000040EDD5DF2E100D0DD6BDD51000142EC34
:1039000004F00601DD2B006E00509EA8FED7AD6EC0
:10391000060EDD5DF2E1DE6B320EDD6F000100DFD1
:1039200001C0DBF60601DBAF05D0DBC6DCF6FF0E1F
:10393000016E36D0DD6BDD51000158EC04F006015C
:10394000DD2B006E00509EA8FED7AD6E040EDD5D2F
:10395000F2E1020EDD6FFA0EEB6F0001CCEC10F01D
:103960000601DD2FF8D7AFCFDAF6D9C6AFFF410E8B
:103970009EA8FED7AD6E540E9EA8FED7AD6EDE6B30
:10398000640EDD6F0001CCDE01AE07D0DAC6AFFFFA
:10399000FE0E016E060104D00001000E016E06014C
:1039A0000001E8EF1DF0F2CFDDF6F29CF29EAA6A6C
:1039B000550EA96EA69CA69EA680A8500601DDBD48
:1039C000F28CDDBFF28EDE6FF2CFDFF6F29CF29E5C
:1039D000AA6A540EA96EA69CA69EA680A850DFBD1A
:1039E000F28CDFBFF28EDEC603F0016EDEC602F09F
:1039F0000001000CEACFF4F6E9CFF3F60601ED3949
:103A0000F009EF6FEF27E20FF06F320FF26FED5119
:103A10000F0BF027F027F227E90FF16FF127F127BD
:103A2000EC390F0BF127F227F137F237F21FF2379B
:103A3000EC510F0BF227EF37070EEE6F0A0EF1076E
:103A4000F227FDE3F007F127FDE3EF07F027FDE3A1
:103A5000EE07EF27FDE3060EEA6EEE0EE96E070EA7
:103A6000F315F39DE926F20EE95CD8B4F38DEF501F
:103A7000006E08E1F3BD06D0F3B90CD0F3B702D065
:103A8000200E03D0F387F399300E002600509EA835
:103A9000FED7AD6EEE50F3ADE6D70001000C83DF2C
:103AA00002C0DAF601C0D9F60601DB6BDB5100017A
:103AB000B5EC03F00601DB2B006E00509EA8FED78C
:103AC000AD6E100EDB5DF2E1090EE96EDAC6EDF6C1
:103AD000D9C6ECF600018EDF220E9EA8FED7AD6E91
:103AE0000601DE6B320EDD6F00011ADE0150F1EFD0
:103AF0001DF00601D96BD951000189EC03F00601D4
:103B0000D92B006E00509EA8FED7AD6E090ED95D70
:103B1000F2E1DE6B640EDD6F000102DE0150FF0892
:103B200003E0000E016E00D0F9EF1DF00401B0516A
:103B3000000A000109E0010A43E0030A51E0010A1A
:103B400057E0070A5FE05FD01ED601C0D8F6060135
:103B5000D8BF11D0D82D08D0040ED96F00014AEC7F
:103B600011F0368A06D00601010ED96F00014AEC29
:103B700011F04CD00601AF501A0A000105E0170AF7
:103B800006E05D0A07E009D00D0EAF6E09D0500EB9
:103B9000AF6E06D0A20EAF6E03D01A0EAF6E00D07D
:103BA0000401B12BB151090809E20D0EAF6E040EEC
:103BB0000601D96F00014AEC11F0368A000126D0C7
:103BC000AF500D0806E00D0E0601D96F000137D683
:103BD00006D0020E0601D96F00014AEC11F016D092
:103BE0005ED7030E0601D96F00014AEC11F00ED02A
:103BF00080D701BE06D0040E0601D96F00014AEC41
:103C000011F004D003D08DEC11F000D0BEEF4AF0DB
:103C10000401B051040803E1010E016E02D0000E50
:103C2000016E0001C2EF4AF0D9C603F00601D8C602
:103C3000E9FFD9C6EAFFEF50430803E0000E016E2A
:103C40004DD0010ED825016E000ED921036E01C0A2
:103C5000E9FFEA6EEF504C0803E0000E016E3ED023
:103C6000020ED825016E000ED921036E01C0E9FFB6
:103C7000EA6EEF50490803E0000E016E2FD0030EEC
:103C8000D825016E000ED921036E01C0E9FFEA6E4E
:103C9000EF50450803E0000E016E20D0040ED82539
:103CA000016E000ED921036E01C0E9FFEA6EEF50EC
:103CB0004E0803E0000E016E11D0050ED825016EEE
:103CC000000ED921036E01C0E9FFEA6EEF505408DF
:103CD00003E0000E016E02D0010E016E00017CEFC8
:103CE0001FF0D9C603F00601D8C6E9FFD9C6EAFF1E
:103CF000EF50430803E0000E016E5CD0010ED825A2
:103D0000016E000ED921036E01C0E9FFEA6EEF508B
:103D10004F0803E0000E016E4DD0020ED825016E53
:103D2000000ED921036E01C0E9FFEA6EEF504E0884
:103D300003E0000E016E3ED0030ED825016E000E8A
:103D4000D921036E01C0E9FFEA6EEF504E0803E08F
:103D5000000E016E2FD0040ED825016E000ED92161
:103D6000036E01C0E9FFEA6EEF50450803E0000E64
:103D7000016E20D0050ED825016E000ED921036EEC
:103D800001C0E9FFEA6EEF50430803E0000E016E48
:103D900011D0060ED825016E000ED921036E01C088
:103DA000E9FFEA6EEF50540803E0000E016E02D006
:103DB000010E016E000194EF1FF0D9C603F0060159
:103DC000D8C6E9FFD9C6EAFFEF50440803E0000E69
:103DD000016E89D0010ED825016E000ED921036E27
:103DE00001C0E9FFEA6EEF50490803E0000E016EE2
:103DF0007AD0020ED825016E000ED921036E01C0C3
:103E0000E9FFEA6EEF50530803E0000E016E6BD03D
:103E1000030ED825016E000ED921036E01C0E9FF03
:103E2000EA6EEF50430803E0000E016E5CD0040E12
:103E3000D825016E000ED921036E01C0E9FFEA6E9C
:103E4000EF504F0803E0000E016E4DD0050ED8254F
:103E5000016E000ED921036E01C0E9FFEA6EEF503A
:103E60004E0803E0000E016E3ED0060ED825016E0E
:103E7000000ED921036E01C0E9FFEA6EEF504E0833
:103E800003E0000E016E2FD0070ED825016E000E44
:103E9000D921036E01C0E9FFEA6EEF50450803E047
:103EA000000E016E20D0080ED825016E000ED9211B
:103EB000036E01C0E9FFEA6EEF50430803E0000E15
:103EC000016E11D0090ED825016E000ED921036EA6
:103ED00001C0E9FFEA6EEF50540803E0000E016EE6
:103EE00002D0010E016E0001A1EF1FF00601D96B97
:103EF0003F0ED86F000198D6015203E0000E016E0C
:103F000029D00601E06B3F0EDF6F000143EC1BF090
:103F1000015204E03688000E016E1CD00601D96BF8
:103F20003F0ED86F0001DDD6015205E0368A369883
:103F3000000E016E0FD00601D96B3F0ED86F000145
:103F40003CD7015205E0369A3698000E016E02D039
:103F5000FF0E016E92EF49F0DAC6DCF6D9C6DBF649
:103F6000DCC603F00601DBC6E9FFDCC6EAFFEF5260
:103F700006E0DB2BD8B4DC2B0001F2D70601D951C7
:103F8000DB5D006EDA51DC59036E00C001F0026E99
:103F90000001000C0601DF5342E0DBC6E9FFDCC68E
:103FA000EAFFEFCFE0F6DEC603F0DDC6E9FFDEC6CE
:103FB000EAFFEF50E05D18E0DCC603F0DBC6E9FF86
:103FC000DCC6EAFFEFCFE0F6DEC603F0DDC6E9FFB0
:103FD000DEC6EAFFEF50E05D03E2FF0E036E01D0A4
:103FE000010E016E1ED00BD0DCC603F0DBC6E9FF6C
:103FF000DCC6EAFFEF5203E1000E016E12D0DCC610
:1040000003F0DB51DB2BD8B4DC2BDEC603F0DD5133
:10401000DD2BD8B4DE2BDF070001BCD70601000E74
:10402000016E0001000C0601F551F703F3CF01F01A
:10403000F4CF00F0F803F3500026F651F703F350E5
:104040000020026E0001000C0601E36BE16B0A0E1A
:10405000E26FE06BDF6BDD51DE1104E1000E016EFB
:10406000026EE4D0E351E32B036ADD25E96EDE51F5
:104070000320EA6EEFCFE4F6E4512D080DE1010EC6
:10408000E16FE351E32B036ADD25E96EDE51032086
:10409000EA6EEFCFE4F60DD0E4512B080AE1E351CC
:1040A000E32B036ADD25E96EDE510320EA6EEFCFD4
:1040B000E4F6E4512F08D8B0ABD0E4513908D8A0C9
:1040C000A7D0E451300821E1036AE351DD25E96E10
:1040D000DE510320EA6EEF5078080AE0036AE351EC
:1040E000DD25E96EDE510320EA6EEF5058080DE140
:1040F000100EE26FE32BE351E32B036ADD25E96E3B
:10410000DE510320EA6EEFCFE4F6E2510A0823E124
:10411000E4512F081FE2E45139081CE3F66B0A0E44
:10412000F56FE0C6F8F6DFC6F7F600017CDF300E6B
:104130000601E45D0124DF6F000E0220E06FE35111
:10414000E32B036ADD25E96EDE510320EA6EEFCF33
:10415000E4F6DED75DD0E25110085AE1E451600880
:1041600006E2E4517A0803E3E451DF0B01D0E451A5
:10417000E46FE4512F0803E2E451390806E2E45108
:10418000400846E2E451460843E3E4512F0817E2B1
:10419000E451390814E3DF35E56FE035E66FE537C4
:1041A000E637E537E637E537E637F00EE517300E48
:1041B000E45DE525DF6F000EE621E06F14D0DF350A
:1041C000E56FE035E66FE537E637E537E637E537A3
:1041D000E637F00EE517410EE45D0A0FE525DF6FC7
:1041E000000EE621E06FE351E32B036ADD25E96E63
:1041F000DE510320EA6EEF50E46F600806E2E451FE
:104200007A0803E3E451DF0B01D0E451E46FB1D746
:10421000E2510A0807E1E12D05D0DF1FE01FDF2B87
:10422000D8B4E02BDFC601F0E0C602F00001000CBC
:10423000040157C401F00001000C0601E951010816
:1042400003E2FF0E016E40D0000174EC13F0015246
:1042500004E0FF0E016E060137D0010E0601F66F75
:10426000000146EC10F087940601E751010A0001B5
:1042700003E0030A08E00ED0840E0601F86F000187
:104280007FEC10F00BD0870E0601F86F00017FEC79
:1042900010F004D0FF0E016E060116D0FF0E0601CD
:1042A000F86F00017FEC10F0E9C6F8F67FEC10F033
:1042B000E8C6F8F67FEC10F0E6C6F8F67FEC10F0F2
:1042C0008784000E016E06010001000CE8C659F457
:1042D000E7C658F40601E8510F0803E2FF0E016E2D
:1042E00042D0000174EC13F0015204E0FF0E016EA5
:1042F000060139D0010E0601F66F000146EC10F000
:1043000087940601E651010A000103E0030A08E070
:104310000ED0830E0601F86F00017FEC10F00CD078
:10432000860E0601F86F00017FEC10F005D0FE0E3E
:10433000016E060118D00001D8900601E737E83772
:10434000E8C6F8F600017FEC10F0E7C6F8F67FEC5F
:1043500010F0FF0E0601F86F00017FEC10F087846B
:10436000000E016E060100012FEF22F00601E75159
:10437000886E956A8492E86BE8513F0818E3E6512D
:10438000C00BE825856EE851E425016E000EE5219D
:1043900001C0E9FFEA6EEFCF8CFF849400000000BB
:1043A00000000000000000008484E82BE5D7848230
:1043B000FF0E956E00017FEF22F03ADF012C55D001
:1043C0009DC4E4F604019E51010B0601E56FE2C6AF
:1043D000E6F6010EE76FE5C6E9F69DC4E8F60001D2
:1043E0002CDF0601E35322E09DC4E4F604019E5154
:1043F000010B0601E56FE43D03D0E52D01D016D099
:1044000004019D2BD8B49E2B9DC4E4F604019E515B
:10441000010B0601E56FE66B010EE76FE5C6E9F6F5
:104420009DC4E8F6000109DF0601DED79DC4E4F66D
:1044300004019E51010B0601E56FE43D10D0E52D0E
:104440000ED0D890E56B04019E310601E46F010E99
:10445000E66FE5C6E8F6E4C6E7F6000137D70401E3
:104460009D2BD8B49E2B54D0000104019D513F0BCD
:104470000601E46FE56B5B0EE425E96E040EE521B1
:10448000EA6EE2C6EFFFE3531CE004019D513F0BCF
:104490000601E46FE56BE4513F0802E1E55311E0EA
:1044A00004019D2BD8B49E2B9D513F0B0601E46F58
:1044B000E56B5B0EE425E96E040EE521EA6EEF6A1A
:1044C000E4D704019D513F0B0601E46FE56BE45115
:1044D0003F081AE1E55318E104015A53D8B402D059
:1044E0000601FAD7878E9D9A040E0601E56F5B0ED2
:1044F000E46F9EC4E7F69DC4E6F6000137D79D8AB7
:10450000879E020E04015A6F04019D2BD8B49E2B86
:104510000001000C0601DA51DBC6E0F6DAC6DFF670
:1045200005019B510601E05D0DE308E1DF51050146
:104530009A5DD8A002D0060105D00601E0C69BF521
:10454000DFC69AF5D9C6DEF6D8C6DDF6DEC6E2F6D7
:10455000E36B000132DFDDC6E2F60601E36B00012A
:104560002CDFDBC6DEF6DAC6DDF6DEC6E2F60601D5
:10457000E36B000122DFDDC6E2F6DCC6E3F61DDFF9
:10458000D9C69FF5D8C69EF5DBC6A1F5DAC6A0F55B
:104590000501982BD8B4992B0001000CDCC6DEF67F
:1045A000DBC6DDF6AA6ADAC6A9FFDDC6A8FFA69CAF
:1045B000A69EA684F2CF00F0F29CF29E0F01550E4B
:1045C000A76EAA0EA76EA682A6B2FED7A69400502A
:1045D000F212010E0601DA25DF6FAA6AA96EDEC6A5
:1045E000A8FFA69CA69EA684F2CF00F0F29CF29EA5
:1045F0000F01550EA76EAA0EA76EA682A6B2FED711
:10460000A6940050F2120001000C9DC5D9F69CC57D
:10461000D8F6A1C5DBF6A0C5DAF6010E0601DC6FFF
:10462000000178DF020E0601DA6F9BC5DCF69AC541
:10463000DBF60001B3DF040E0601DA6F9DC5DCF680
:104640009CC5DBF60001AADF060E0601DA6F99C5EC
:10465000DCF698C5DBF60001A1DF0501976B966BD0
:10466000956B946B0601D96B0001A1EC11F0000C65
:104670004550730807E14650310804E10501976B86
:10468000966B00014750440805E14850310802E1AB
:10469000368C01D0369C4950700816E10601DE6B5D
:1046A0004A0EDD6F0001D0DC02C089F501C088F53B
:1046B00005018951070807E2FF0A03E18851FC0858
:1046C00002E2896B886B000143504C0804E14450BE
:1046D000320801E19ADF7DEF2AF0F2CFDBF6F29C9F
:1046E000F29EAA6A010EA96EA69CA69EA680A8505C
:1046F0000601DBBDF28CDBBFF28E016E000189EF9B
:1047000023F00501932D03D0010E016E0CD00001A2
:10471000E4D7015205E0020E016E050104D000014C
:10472000000E016E05010001EEEF24F0200E0601DF
:10473000DEA9300EDF6FDDC600F0DDAF07D0001E52
:10474000002A00C0DDF62D0EDF6FDE8F0150DDC6C2
:10475000E5F6640EE66F00015CEC15F000C0DDF6D6
:10476000300E01240601E06FDDC6E5F60A0EE66FA5
:1047700000015CEC15F0300E00240601E26F300EF3
:104780000124E16FDFC600F0DEA702D0DEAFDE95C8
:10479000DEB90BD0DEAF22D0DEB520D000C0E0F60F
:1047A000DEB31CD000C0E1F619D0300EE05D16E19A
:1047B00000C0E0F6200EDF6FDEA704D0DE95DE83BA
:1047C000DEAFDE93300EE15D09E100C0E1F6200EC0
:1047D000E06FDEA7F7D7DE93DEAFDE91DEA504D073
:1047E000DF519EA8FED7AD6EDEA304D0E0519EA897
:1047F000FED7AD6EDEA104D0E1519EA8FED7AD6E0E
:10480000E2519EA8FED7AD6E0001000C016A026A5B
:10481000006A036A0601F85102E1F75118E0100E30
:10482000F96FD890F537F63700360336F851035C48
:1048300002E1F751005C07E3F751005ED8A00306E0
:10484000F851035ED88001360236F92FEAD700000E
:104850000001000CEACFECF6E9CFEBF60601E5AF7C
:1048600008D0EB8FEBA9EB2BE41FE51FE42BD8B4AA
:10487000E52BE539F009E76FE727E20FE86F320F24
:10488000EA6FE5510F0BE827E827EA27E90FE96F00
:10489000E927E927E4390F0BE927EA27E937EA375F
:1048A000EA1FEA37E4510F0BEA27E737070EE66FF6
:1048B0000A0EE907EA27FDE3E807E927FDE3E70732
:1048C000E827FDE3E607E727FDE3060EEA6EE60EBE
:1048D000E96E070EEB15EB9DE906EB1507E1EBB969
:1048E000E92AEBB903D0200E006E1CD0E926EA0EAF
:1048F000E95CD8B4EB8DEF50006E08E1EBBD06D05B
:10490000EBB914D0EBB702D0200E0BD0EBAF06D032
:104910002D0E006EED50EB9DEB9F04D0EB87EB99D5
:10492000300E002600509EA8FED7AD6EEE50EBADC7
:10493000DED70001000C050109C501F00AC502F02F
:104940000001FDEF25F00601DB6BDB5107082CE3CE
:104950004C0EDB25F2CFDEF6F29CF29EAA6AA96E1F
:10496000A69CA69EA680A850DEBDF28CDEBFF28E6D
:10497000DC6FDC512F0803E2DC5139080AE2036ADC
:10498000DB51440FE96E040E0320EA6E300EEF6E29
:1049900009D0036ADB51440FE96E040E0320EA6E6E
:1049A000DCC6EFFFDB2BD1D704014C6B440E016E4C
:1049B000040E026E0001000C0601DB6BDB510001EE
:1049C0007DEC05F00601DB2B006E00509EA8FED7A3
:1049D000AD6E040EDB5DF2E1000193D601C0D8F6A6
:1049E0004C0E9EA8FED7AD6ED8C6DDF61F0E060192
:1049F000DE6F00019BDE99C5DAF698C5D9F6720E16
:104A00009EA8FED7AD6E000EE96EDAC6EDF6D9C6E9
:104A1000ECF6FAEC1CF095C5DAF694C5D9F6DAC6D0
:104A2000F6F6D9C6F5F60E0E0601F86F100EF76F02
:104A30000001ECDE02C0DCF601C0DBF602C0F6F6D7
:104A400001C0F5F60601F86B180EF76F0001DEDE07
:104A500000C0DCF6060103C0DDF6DAC6F6F6D9C6FC
:104A6000F5F6F86B3C0EF76F0001D0DE02C0DFF602
:104A700001C0DEF602C0F6F601C0F5F60601F86BDD
:104A80003C0EF76F0001C2DE00C0DFF6060103C076
:104A9000E0F6DAC6F6F6D9C6F5F6F86B3C0EF76F17
:104AA0000001B4DE00C0E1F6060103C0E2F6650EC7
:104AB0009EA8FED7AD6E040EE96EDDC6EDF6DCC62F
:104AC000ECF60001FAEC1CF03A0E9EA8FED7AD6E93
:104AD0000B0EE96EE0C6EDF6DFC6ECF6FAEC1CF064
:104AE0003A0E9EA8FED7AD6E0B0EE96EE2C6EDF64D
:104AF000E1C6ECF6FAEC1CF097C5DAF696C5D9F6E5
:104B0000DAC6F6F6D9C6F5F60E0E0601F86F100EE7
:104B1000F76F00017BDE02C0DCF601C0DBF602C0ED
:104B2000F6F601C0F5F60601F86B180EF76F0001F6
:104B30006DDE00C0DCF6060103C0DDF6DAC6F6F66F
:104B4000D9C6F5F6F86B3C0EF76F00015FDE02C0C8
:104B5000DFF601C0DEF602C0F6F601C0F5F606018A
:104B6000F86B3C0EF76F000151DE00C0DFF6060166
:104B700003C0E0F6DAC6F6F6D9C6F5F6F86B3C0ED9
:104B8000F76F000143DE00C0E1F6060103C0E2F664
:104B9000730E9EA8FED7AD6E040EE96EDDC6EDF66F
:104BA000DCC6ECF60001FAEC1CF03A0E9EA8FED72B
:104BB000AD6E0B0EE96EE0C6EDF6DFC6ECF6FAEC74
:104BC0001CF03A0E9EA8FED7AD6E0B0EE96EE2C643
:104BD000EDF6E1C6ECF6FAEC1CF087C5DAF686C510
:104BE000D9F6700E9EA8FED7AD6E0A0EE96EDAC633
:104BF000E5F6D9C6E4F62EDE9ED602C0DAF601C08E
:104C0000D9F6740E9EA8FED7AD6E0B0EE96EDAC60D
:104C1000E5F6D9C6E4F61EDE355203E13450190834
:104C200009E2540E9EA8FED7AD6E310E9EA8FED7A7
:104C3000AD6E08D0540E9EA8FED7AD6E300E9EA865
:104C4000FED7AD6E8FC5D8F6620E9EA8FED7AD6EAC
:104C5000D8C6DDF6130E0601DE6F000167DDD3EC6A
:104C60001CF002C0DAF601C0D9F60601DB6BDB519D
:104C7000000192EC05F00601DB2B006E00509EA8AF
:104C8000FED7AD6E060EDB5DF2E1090EE96EDAC607
:104C9000EDF6D9C6ECF60001FAEC1CF0200E9EA849
:104CA000FED7AD6E0601DB6BDB510001ABEC05F00E
:104CB000000907E00601DB2B9EA8FED7AD6EF4D7F6
:104CC0000001570E9EA8FED7AD6E4C0E9EA8FED7D3
:104CD000AD6E39DE02C0DCF601C0DBF6630E9EA8C5
:104CE000FED7AD6EDCC6EAFFDBC6E9FF000EEF10B3
:104CF00008E09EA8FED7EFCFADFFE92AD8B4EA2A94
:104D0000F5D70D0E9EA8FED7AD6E0A0E9EA8FED753
:104D1000AD6E0A0E386E000C04019E6B9D6B000197
:104D2000000C500E0601E26FE36B0001DDEC21F098
:104D3000770E0601E26FE36B0001DDEC21F0060166
:104D4000D96B020ED86FD95103081CE33F0ED8254A
:104D5000E96E000ED921EA6EEF5201E113D03F0E49
:104D6000D825E96E000ED921EA6EEFCFDAF6DAC661
:104D7000E2F6E36B0001DDEC21F00601D82BD8B49C
:104D8000D92BE1D7E26B010EE36F0001DDEC21F0DE
:104D9000000CE4C69CF4E3C69BF4000C74EC13F026
:104DA000015203E0000E016E4AD0010E0601F66FBB
:104DB000000146EC10F08794D20E0601F86F000156
:104DC0007FEC10F0E4C600F0E5C601F0026A036A69
:104DD000E4C6E8F6E4C6F8F67FEC10F0E3C600F0AF
:104DE000E4C601F0E5C602F0036AE3C6E8F6E3C6EE
:104DF000F8F67FEC10F0E2C6F8F67FEC10F0FF0E4C
:104E00000601F86F00017FEC10F0FF0E0601F86F4D
:104E100000017FEC10F0FF0E0601F86F00017FEC3F
:104E200010F0FF0E0601F86F00017FEC10F087EC28
:104E300010F001C0E6F687840601E6C601F0000125
:104E400039EF27F004015A5306E00A0E0601EB6F12
:104E50000001CCEC10F0000118EC21F0012C0CD07A
:104E60000601E56BE46B9CC4E3F69BC4E2F600012B
:104E700095D701C0E1F608D09CC4E3F69BC4E2F6E6
:104E800077EC14F001C0E1F604019B2BD8B49C2B05
:104E90000601E1C601F00001000CDBC6E4F6DAC64B
:104EA000E3F677DF0601DD6BDC6BDD51030815E30C
:104EB0000001C8DF01C0DEF60601DE5301E10DD0BE
:104EC00081B2FED7DE517F0BDF6FDF519EA8FED788
:104ED000AD6EDC2BD8B4DD2BE8D70D0E9EA8FED727
:104EE000AD6E0A0E9EA8FED7AD6E0001000C040147
:104EF0009DC401F09EC402F00001000CF2CFE0F668
:104F0000F29CF29EAA6ADDC6A9FFA69CA69EA68078
:104F1000A8500601E0BDF28CE0BFF28EDE6F010EFC
:104F2000DD25F2CFE1F6F29CF29EAA6AA96EA69C5C
:104F3000A69EA680A850E1BDF28CE1BFF28EDF6F85
:104F4000DEC601F0DFC602F00001000C010E060112
:104F5000D96F0001A1EC11F036AC04D0A3C587F5E0
:104F6000A2C586F505019B6B9A6B9D6B9C6B996B3B
:104F7000986B010E0601DD6F00016CEC18F09DC509
:104F8000D9F69CC5D8F687C5DBF686C5DAF60601E4
:104F9000DC6B00018AEC22F0140E0501926F000117
:104FA00068EF2BF0F2CFF1F6F29CF29EAA6A420E65
:104FB000A96EA69CA69EA680A8500601F1BDF28C03
:104FC000F1BFF28EEF6FF2CFF1F6F29CF29EAA6A79
:104FD000430EA96EA69CA69EA680A850F1BDF28C99
:104FE000F1BFF28EF06FF0C603F0EFC601F0F0C62D
:104FF00002F00001000C0601DD6BDD510001C0EC88
:1050000005F00601DD2B006E00509EA8FED7AD6EA8
:10501000040EDD5DF2E1355203E13450190809E276
:105020004C0E9EA8FED7AD6E500E9EA8FED7AD6E5C
:1050300008D04C0E9EA8FED7AD6E300E9EA8FED7AF
:10504000AD6E85C5D9F684C5D8F6700E9EA8FED77C
:10505000AD6E020EE96ED9C6E5F6D8C6E4F60001DB
:105060002AEC24F09FDF02C0D9F601C0D8F6630E07
:105070009EA8FED7AD6E000EE96ED9C6EDF6D8C675
:10508000ECF6FAEC1CF0740E9EA8FED7AD6E030E83
:105090000601DD6F300E9EA8FED7AD6EDD2FFAD76C
:1050A0008DC5DCF68CC5DBF6430E9EA8FED7AD6E33
:1050B000010EE96EDCC6E5F6DBC6E4F600012AEC7B
:1050C00024F08FC5DAF6620E9EA8FED7AD6EDAC662
:1050D000DDF6130E0601DE6F000196EC23F0D3EC33
:1050E0001CF002C0DEF601C0DDF60601DF6BDF5109
:1050F000000192EC05F00601DF2B006E00509EA827
:10510000FED7AD6E060EDF5DF2E1090EE96EDEC67A
:10511000EDF6DDC6ECF60001FAEC1CF0200E9EA8C0
:10512000FED7AD6E0601DD6BDD510001ABEC05F085
:10513000000907E00601DD2B9EA8FED7AD6EF4D76F
:105140000001570E9EA8FED7AD6E4C0E9EA8FED74E
:10515000AD6E0D0E9EA8FED7AD6E0A0E9EA8FED7B0
:10516000AD6E0A0E386E000C0601EC51400A0001CB
:1051700011E0020A13E0060A15E0020A17E00E0A1F
:1051800019E0010A1BE0050A1DE0180A1FE01F0ACA
:1051900021E025D0020E0601ED6F23D0020E06019C
:1051A000ED6F1FD0020E0601ED6F1BD0020E06013F
:1051B000ED6F17D0010E0601ED6F13D0020E060140
:1051C000ED6F0FD0080E0601ED6F0BD0020E060139
:1051D000ED6F07D0010E0601ED6F03D0000154D032
:1051E0000601EE6BED51EE5D4FE2EE51EC25EF6FF7
:1051F000EE51EA25016E000EEB21036E01C0E9FFBE
:10520000EA6EEFCFF0F6AA6AEFC6A9FFF0C6A8FFD4
:10521000A69CA69EA684F2CF00F0F29CF29E0F01FF
:10522000550EA76EAA0EA76EA682A6B2FED7A694AA
:105230000050F2120601EE51EC25160FF06FEE5100
:10524000EA25016E000EEB21036E01C0E9FFEA6E54
:10525000EF50FF0AF16FAA6AF0C6A9FFA86EA69CDC
:10526000A69EA684F2CF00F0F29CF29E0F01550E8E
:10527000A76EAA0EA76EA682A6B2FED7A69400506D
:10528000F2120601EE2BAED70001000C060E06014D
:10529000EB6FE20EEA6F420EEC6F000165DF000C6F
:1052A000020E0601DD6F000129DE02C09BF501C080
:1052B0009AF5040E0601DD6F000120DE02C09DF5A7
:1052C00001C09CF5060E0601DD6F000117DE02C06D
:1052D00099F501C098F50601D86BD851000132EC60
:1052E00005F00601D82B006E00509EA8FED7AD6ECB
:1052F000070ED85DF2E1020EE96E9BC5E5F69AC590
:10530000E4F600012AEC24F06D0E9EA8FED7AD6EE7
:10531000740E9EA8FED7AD6E000EE96E9DC5EDF62B
:105320009CC5ECF6FAEC1CF06E0E9EA8FED7AD6E96
:10533000700E9EA8FED7AD6E000EE96E99C5EDF613
:1053400098C5ECF6FAEC1CF0170E0601D96FD9518E
:10535000000132EC05F00601D92B006E00509EA82A
:10536000FED7AD6E1C0ED95DF2E10A0E386E00015B
:10537000FAEF2BF00601DE6B440EDD6F000124EC2A
:1053800020F002C0DBF601C0DAF6140E0601DD6F74
:105390000001B4DD02C0DEF601C0DDF6DBC6F6F6C4
:1053A000DAC6F5F60601F86B640EF76F000113EC30
:1053B00020F002C0E0F601C0DFF606010134026E03
:1053C000E035036E02360336FC0E02160250DD2570
:1053D000E16F0350DE21E26FE46FE1C6E3F6000106
:1053E000D8DC0601DD6BDD51000153EC05F0060150
:1053F000DD2B006E00509EA8FED7AD6E050EDD5D64
:10540000F2E1D96BD86BD95347E1D851630844E333
:10541000000118DD01C0DCF6DCC6EDF6370E060132
:10542000EE6F000139EC15F00DDD01C0DCF6DCC6D5
:10543000EDF6370E0601EE6F000139EC15F002DDD6
:1054400001C0DCF6DCC6EDF6370E0601EE6F00019A
:1054500039EC15F0F7DC01C0DCF6DCC6EDF6370EF2
:105460000601EE6F000139EC15F005019851D8B432
:105470009907980798530AE1995308E10601DD6BF3
:1054800000016CEC18F0060107D0050104000601CC
:10549000D82BD8B4D92BB7D7DD6BDD51000168EC20
:1054A00005F00601DD2B006E00509EA8FED7AD6E04
:1054B000050EDD5DF2E10A0E386E000119EF2CF0E9
:1054C000050E0601DA6FA40ED96F0001ACEC1FF0D7
:1054D00002C0D9F601C0D8F60601DC6B3F0EDB6FC7
:1054E000050EDE6FA40EDD6F01C0DFF60001CAEC11
:1054F0001FF0015207E138EF23F0DCEC24F0000E3E
:10550000016EE7D1050E0601DA6FA90ED96F000111
:10551000ACEC1FF002C0D9F601C0D8F60601DC6B76
:105520003F0EDB6F050EDE6FA90EDD6F01C0DFF6EB
:105530000001CAEC1FF0015209E18CEC26F091EC5D
:1055400026F0DCEC24F0000E016EC3D1050E06013E
:10555000DA6FAF0ED96F0001ACEC1FF002C0D9F6C4
:1055600001C0D8F60601DC6B3F0EDB6F050EDE6F67
:10557000AF0EDD6F01C0DFF60001CAEC1FF0015273
:1055800008E10601DB6BDA6B000187DC000E016EBF
:10559000A0D1050E0601DA6FB40ED96F0001ACEC94
:1055A0001FF002C0D9F601C0D8F60601DC6B3F0E31
:1055B000DB6F050EDE6FB40EDD6F01C0DFF600019C
:1055C000CAEC1FF0015216E192DC02C0D9F601C00C
:1055D000D8F6100E0601DA6F02C0DCF601C0DBF669
:1055E0000001CEEC22F091EC26F0DCEC24F0000E71
:1055F000016E6FD1050E0601DA6FBA0ED96F000188
:10560000ACEC1FF002C0D9F601C0D8F60601DC6B85
:105610003F0EDB6F050EDE6FBA0EDD6F01C0DFF6E9
:105620000001CAEC1FF0015211E1100E0601DD6FFE
:10563000000164DC02C0D9F601C0D8F602C0DBF676
:1056400001C0DAF62ADC000E016E43D1050E060118
:10565000DA6FBF0ED96F0001ACEC1FF002C0D9F6B3
:1056600001C0D8F60601DC6B3F0EDB6F050EDE6F66
:10567000BF0EDD6F01C0DFF60001CAEC1FF0015262
:105680002CE135DC02C0D9F601C0D8F6120E0601B5
:10569000DA6F02C0DCF601C0DBF60001CEEC22F0CE
:1056A00091EC26F024DC02C0D9F601C0D8F6140E25
:1056B0000601DA6F02C0DCF601C0DBF60001CEECB9
:1056C00022F00501976B966B956B946B00013ED4AD
:1056D000DCEC24F0000E016EFCD0050E0601DA6F42
:1056E000C50ED96F0001ACEC1FF002C0D9F601C0A5
:1056F000D8F60601DC6B3F0EDB6F050EDE6FC50EC4
:10570000DD6F01C0DFF60001CAEC1FF0015213E1AA
:10571000120E0601DD6F00017EEC27F002C0D9F603
:1057200001C0D8F602C0DBF601C0DAF64DEC27F076
:10573000000E016ECED0050E0601DA6FCA0ED96FCB
:105740000001ACEC1FF002C0D9F601C0D8F606018A
:10575000DC6B3F0EDB6F050EDE6FCA0EDD6F01C026
:10576000DFF60001CAEC1FF0015204E144DC000E38
:10577000016EAFD0050E0601DA6FCF0ED96F0001B2
:10578000ACEC1FF002C0D9F601C0D8F60601DC6B04
:105790003F0EDB6F050EDE6FCF0EDD6F01C0DFF653
:1057A0000001CAEC1FF0015209E185C5E3F684C58A
:1057B000E2F66CDD20DC000E016E8BD0050E0601DA
:1057C000DA6FD40ED96F0001ACEC1FF002C0D9F62D
:1057D00001C0D8F60601DC6B3F0EDB6F050EDE6FF5
:1057E000D40EDD6F01C0DFF60001CAEC1FF00152DC
:1057F00004E156D5000E016E6CD0050E0601DA6F7D
:10580000D90ED96F0001ACEC1FF002C0D9F601C06F
:10581000D8F60601DC6B3F0EDB6F050EDE6FD90E8E
:10582000DD6F01C0DFF60001CAEC1FF0015204E198
:10583000A1D5000E016E4DD0050E0601DA6FDE0E09
:10584000D96F0001ACEC1FF002C0D9F601C0D8F648
:105850000601DC6B3F0EDB6F050EDE6FDE0EDD6FCB
:1058600001C0DFF60001CAEC1FF001520AE1060197
:10587000DD6B00016CEC18F0FBEC27F0000E016E04
:1058800028D0050E0601DA6FE60ED96F0001ACECE8
:105890001FF002C0D9F601C0D8F60601DC6B3F0E3E
:1058A000DB6F050EDE6FE60EDD6F01C0DFF6000177
:1058B000CAEC1FF001520BE1010E0601DD6F000181
:1058C0006CEC18F0FBEC27F0000E016E02D0FF0E1E
:1058D000016E97EF49F0D190879087929D9AF29A46
:1058E000879C320E0601EB6F0001CCEC10F0FFD765
:1058F000000CF2CFF1F6F29CF29EAA6A400EA96E5D
:10590000A69CA69EA680A8500601F1BDF28CF1BF10
:10591000F28EEF6FF2CFF1F6F29CF29EAA6A410E80
:10592000A96EA69CA69EA680A850F1BDF28CF1BFE0
:10593000F28EF06FF0C603F0EFC601F0F0C602F091
:105940000001000CF2CFF7F6F29CF29EAA6A460E16
:10595000A96EA69CA69EA680A8500601F7BDF28C53
:10596000F7BFF28EF56FF2CFF7F6F29CF29EAA6ABD
:10597000470EA96EA69CA69EA680A850F7BDF28CE5
:10598000F7BFF28EF66FF6C603F0F5C601F0F6C665
:1059900002F00001000CF2CFF7F6F29CF29EAA6A28
:1059A000440EA96EA69CA69EA680A8500601F7BD2F
:1059B000F28CF7BFF28EF56FF2CFF7F6F29CF29E03
:1059C000AA6A450EA96EA69CA69EA680A850F7BD01
:1059D000F28CF7BFF28EF66FF6C603F0F5C601F053
:1059E000F6C602F00001000C290E0601D96F2D0E3B
:1059F0009EA8FED7AD6ED92FFAD70A0E9EA8FED765
:105A0000AD6E0D0E9EA8FED7AD6E0A0ED96F2D0E8F
:105A10009EA8FED7AD6ED92FFAD7DA6BDA51000106
:105A20000BEC07F00601DA2B006E00509EA8FED7A3
:105A3000AD6E150EDA5DF2E10A0EDB6F2D0E9EA83B
:105A4000FED7AD6EDB2FFAD70A0E9EA8FED7AD6E3D
:105A50000D0E9EA8FED7AD6E290ED96F2D0E9EA8F5
:105A6000FED7AD6ED92FFAD70A0E9EA8FED7AD6E1F
:105A70000D0E9EA8FED7AD6E0A0E9EA8FED7AD6E87
:105A80000D0E9EA8FED7AD6ED96BD951000104EC66
:105A900006F00601D92B006E00509EA8FED7AD6E11
:105AA000090ED95DF2E1DA6BDA510001ABEC05F0D9
:105AB000000906E00601DA2B9EA8FED7AD6EF4D7EA
:105AC0000B0E0601DB6FDB51000104EC06F0060152
:105AD000DB2B006E00509EA8FED7AD6E0F0EDB5D77
:105AE000F2E10001D3EC1CF002C0DAF601C0D9F6F5
:105AF0000601DB6BDB51000129EC07F00601DB2B13
:105B0000006E00509EA8FED7AD6E120EDB5DF2E176
:105B1000090EE96EDAC6EDF6D9C6ECF60001FAEC2C
:105B20001CF00A0E9EA8FED7AD6E0D0E9EA8FED7E5
:105B3000AD6ED2EC27F002C0DAF601C0D9F606014C
:105B4000DB6BDB51000148EC07F00601DB2B006E3C
:105B500000509EA8FED7AD6E0D0EDB5DF2E1100E7B
:105B6000E96EDAC6EDF6D9C6ECF60001FAEC1CF0E7
:105B70000A0E9EA8FED7AD6E0D0E9EA8FED7AD6E86
:105B8000B8DE02C0DAF601C0D9F60601DB6BDB51E4
:105B9000000164EC07F00601DB2B006E00509EA8AC
:105BA000FED7AD6E0D0EDB5DF2E1100EE96EDAC6CA
:105BB000EDF6D9C6ECF60001FAEC1CF00A0E9EA830
:105BC000FED7AD6E0D0E9EA8FED7AD6EBBDE02C039
:105BD000DAF601C0D9F60601DB6BDB51000180EC7F
:105BE00007F00601DB2B006E00509EA8FED7AD6EBD
:105BF0000D0EDB5DF2E1100EE96EDAC6E5F6D9C6F0
:105C0000E4F600012AEC24F00A0E9EA8FED7AD6E41
:105C10000D0E9EA8FED7AD6EBEDE02C0DAF601C044
:105C2000D9F60601DB6BDB5100019CEC07F00601A5
:105C3000DB2B006E00509EA8FED7AD6E080EDB5D1C
:105C4000F2E1030EDC6F200E9EA8FED7AD6EDC2FB6
:105C5000FAD73D0E9EA8FED7AD6E200E9EA8FED7A9
:105C6000AD6E100EE96EDAC6EDF6D9C6ECF600019F
:105C7000FAEC1CF00A0E9EA8FED7AD6E0D0E9EA883
:105C8000FED7AD6EA3EC24F002C0DAF601C0D9F65F
:105C90000601DB6BDB510001B6EC07F00601DB2BE4
:105CA000006E00509EA8FED7AD6E0A0EDB5DF2E1DD
:105CB000040EDC6F790E9EA8FED7AD6EDC2FFAD7EE
:105CC0000A0EDD6FDD510001B6EC07F00601DD2B99
:105CD000006E00509EA8FED7AD6E120EDD5DF2E1A3
:105CE000DAC6EAFFD9C6E9FF000EEF1008E09EA869
:105CF000FED7EFCFADFFE92AD8B4EA2AF5D70A0ECE
:105D00009EA8FED7AD6E0D0E9EA8FED7AD6E0A0EF4
:105D10009EA8FED7AD6E0D0E9EA8FED7AD6E070EE7
:105D2000D96F2D0E9EA8FED7AD6ED92FFAD71B0EB8
:105D3000DA6F210E9EA8FED7AD6EDA2FFAD7070EC6
:105D4000DB6F2D0E9EA8FED7AD6EDB2FFAD70A0EA5
:105D50009EA8FED7AD6E0D0E9EA8FED7AD6E070EA7
:105D6000D96F2D0E9EA8FED7AD6ED92FFAD7DA6B5C
:105D7000DA510001D4EC07F00601DA2B006E005076
:105D80009EA8FED7AD6E1B0EDA5DF2E1070EDB6F4B
:105D90002D0E9EA8FED7AD6EDB2FFAD70A0E9EA859
:105DA000FED7AD6E0D0E9EA8FED7AD6E070ED96F55
:105DB0002D0E9EA8FED7AD6ED92FFAD71B0EDA6F27
:105DC000210E9EA8FED7AD6EDA2FFAD7070EDB6F35
:105DD0002D0E9EA8FED7AD6EDB2FFAD70A0E9EA819
:105DE000FED7AD6E0D0E9EA8FED7AD6E0001000C65
:105DF00081B404D0020E0501916F000181B603D079
:105E0000010E0501916F05019151905D07E091C56B
:105E100090F5010E0401B96F2C0EB86F0401B85350
:105E20001EE1B9531CE191C590F505019151000A9D
:105E3000000105E0010A08E0030A0BE00FD0640E40
:105E400005018F6F00010AD0320E05018F6F00012E
:105E500005D0140E05018F6F000100D00401000170
:105E600078EF34F0829087EC10F0036A01C09FF461
:105E7000040103C0A0F49FC4A0F49F6B000187EC51
:105E800010F0015004019F1382809F51FC0B06010A
:105E9000EB6FA0C4ECF60601EB5308E1EC5181086E
:105EA00005E10001BEEC0FF000D0060100015AEF41
:105EB0002FF0D8D70401A031036E9F31026E033258
:105EC0000232033202320332023203320232070E4E
:105ED00003160250AC270350AD23D890AB35036AAC
:105EE000020F016E000E032201509F0FE96E040E97
:105EF0000320EA6EECCF03F0ED52EF50AC5F03509D
:105F0000AD5BD890AB35036A020F016E000E032221
:105F100001509F0FE96E040E0320EA6EA031036E5C
:105F20009F31026E033202320332023203320232F6
:105F300003320232070E031602C0EFFF03C0ECFF6C
:105F4000AB2BAB51040801E2AB6BADC4F6F6ACC4AD
:105F5000F5F60601F86B050EF76F000113EC20F063
:105F600002C0AFF401C0AEF481EF34F0000E0401C2
:105F7000B4B3010E000A01E150D0B493AFC48DF563
:105F8000AEC48CF58CC500F08DC501F0026A036AC1
:105F900001AE02D00206030603C0EEF602C0EDF623
:105FA00001C0ECF600C0EBF6EEC6FCF6EDC6FBF663
:105FB000ECC6FAF6EBC6F9F60701006B0601FF6BBB
:105FC000FE6B880EFD6F00014BEC12F003C0EEF685
:105FD00002C0EDF601C0ECF600C0EBF60601ECC61F
:105FE000EBF6EDC6ECF6EEC6EDF6EE6BEE33ED330A
:105FF000EC33EB33EE33ED33EC33EB33EE33ED33A5
:10600000EC33EB33EE33ED33EC33EB330F0EEE17B3
:10601000ECC68BF5EBC68AF50401000188EF34F07D
:106020000601F781080EF86F00017FEC10F087EC95
:1060300010F001C0F6F60601F6AD03D0FE0E016EBB
:106040003AD0F6AF03D0FF0E016E35D0380EF86FA0
:1060500000017FEC10F00601F66BF651020824E314
:10606000020ED880F655036A4D0F016E040E03220E
:1060700001C0F9F603C0FAF6000187EC10F0FAC689
:10608000EAFFF9C6E9FF01C0EFFF020ED880060162
:10609000F655036A4D0FE96E040E0320EA6EEF52C7
:1060A000D8A4F791F62BD9D7F7A103D0FE0E016E35
:1060B00002D0000E016E0001000C82808282878E69
:1060C0009D9A020E0601F66F000146EC10F08294D4
:1060D000A7DF01C0EFF682849D8A879E0601EFBF8D
:1060E00001D003D0EFC601F041D04FC45EF54EC4DD
:1060F0005DF55DC500F0026A036A00500501802766
:106100005E5181230250822303508323D8907F3530
:10611000036A5F0FE96E050E0320EA6EECCF03F011
:10612000ED52EFCF00F003C001F0026A036A0050A5
:10613000805F0150815B0250825B0350835BD8908B
:106140007F35036A5F0FE96E050E0320EA6E5EC5B8
:10615000ECFFED525DC5EFFF7F2B7F510F0801E291
:106160007F6B0401B481000E016E06010001ECEFAB
:1061700030F082828280020E0601F66F000146EC4A
:1061800010F094948294AAEC10F001BE01D011D0CA
:106190008284140E006E002EFED700008294E2EC82
:1061A00010F08284140E006E002EFED70000829440
:1061B000EAD78284000C36AC05D089C587F588C53E
:1061C00086F5E9D00401B55303E00001E4D00401F1
:1061D000070EB56F000171D70150FF0A03E0010AF5
:1061E00011E016D0010E0401B56FB351640807E247
:1061F0000001BFDF0401B36B0A0EB56F01D0B32BF2
:106200000001C9D00A0E0401B56F0001B2DFC3D08E
:106210000401B36B050183310601EE6F0501823184
:106220000601ED6F050181310601EC6F050180313A
:106230000601EB6FEE33ED33EC33EB33EE33ED333E
:10624000EC33EB33EE33ED33EC33EB330F0EEE1771
:10625000EEC6FCF6EDC6FBF6ECC6FAF6EBC6F9F6B2
:106260000701006B0601FF6B130EFE6F880EFD6FBA
:1062700000014BEC12F003C0EEF602C0EDF601C0D7
:10628000ECF600C0EBF6EDC6EBF6EEC6ECF606015A
:10629000ED6BEE6BECC685F5EBC684F50001D2EC38
:1062A00027F001C000F002C001F0026A036A060193
:1062B000EE51035C11E30BE1ED51025C0DE307E1EC
:1062C000EC51015C09E303E10050EB5D05E20501DF
:1062D000876B866B00015FD00001D2EC27F0015084
:1062E0000601EB5F0250EC5B000EED5BEE5B000124
:1062F00079EC2CF002C0F0F601C0EFF6EACFF2F62E
:10630000E9CFF1F6EEC6FCF6EDC6FBF6ECC6FAF602
:10631000EBC6F9F60701006B0601FF6B02C0FEF643
:1063200001C0FDF600014BEC12F0F2C6EAFFF1C627
:10633000E9FF03C0EEF602C0EDF601C0ECF600C0C6
:10634000EBF60601ECC6EBF6EDC6ECF6EEC6EDF6A6
:10635000EE6BEE33ED33EC33EB33EE33ED33EC3306
:10636000EB33EE33ED33EC33EB33EE33ED33EC3331
:10637000EB33EE33ED33EC33EB33EE33ED33EC3321
:10638000EB33EE33ED33EC33EB33010EEE17ECC6AB
:1063900087F5EBC686F500018BEF34F082848280AE
:1063A000878E9D9A82923CDE01C0F5F682829D8A9C
:1063B000879E0601F5AF03D0F5C601F04BD004016E
:1063C000BD6B4FC4BCF44EC4BBF44DC4BAF4BA5157
:1063D000FF27BB51050100230401BC510501012326
:1063E0000401BD51050102230401FE51040DF350C7
:1063F000036ABE0FE96E040E0320EA6EEFCF00F0D1
:10640000ECCF01F0ECCF02F0ECCF03F00050FF5FD7
:1064100001500501005B0250015B0350025B040167
:10642000FE51040DF350036ABE0FE96E040E032003
:10643000EA6EBAC4EFFFBBC4ECFFBCC4ECFFBDC442
:10644000ECFFFE2BFE510F0801E2FE6B368E000EB4
:10645000016E0601000151EF32F082848280949235
:106460008292AAEC10F001BE01D011D08282140EEB
:10647000006E002EFED700008292E2EC10F08282C5
:10648000140E006E002EFED700008292EAD78282A0
:10649000000C0401B65301E016D2070EB66F0001DE
:1064A0007DD70150FF0A03E0010A11E017D0010E69
:1064B0000401B66FB251640807E20001CEDF0401A7
:1064C000B26B0A0EB66F01D0B22BFDD100010A0EDD
:1064D0000401B66F0001C1DF0401F5D10401B26B04
:1064E000050102310601F46F050101310601F36F68
:1064F000050100310601F26F0401FF310601F16F61
:10650000F433F333F233F133F433F333F233F1335F
:10651000F433F333F233F1330F0EF417F4C6FCF611
:10652000F3C6FBF6F2C6FAF6F1C6F9F60701006B00
:106530000601FF6B030EFE6FE80EFD6F00014BECD2
:1065400012F003C0F4F602C0F3F601C0F2F600C088
:10655000F1F60601F2C6F1F6F3C6F2F6F4C6F3F66A
:10656000F46BF433F333F233F133F433F333F233C4
:10657000F133F433F333F233F133F433F333F233EF
:10658000F133F433F333F233F133F433F333F233DF
:10659000F133030EF417F4C606F5F3C605F5F2C69B
:1065A00004F5F1C603F5F4530AE1F35308E1F2519F
:1065B00012080CE2FF0A03E1F151880807E2030E1A
:1065C00005010A6F090E096F04017DD10001CBECB2
:1065D0002CF002C0F6F601C0F5F6EACFF8F6E9CFE6
:1065E000F7F6F4C6FCF6F3C6FBF6F2C6FAF6F1C609
:1065F000F9F60701006B0601FF6B02C0FEF601C051
:10660000FDF600014BEC12F0F8C6EAFFF7C6E9FF11
:1066100003C0F4F602C0F3F601C0F2F600C0F1F6D2
:10662000F2C607F5F3C608F505018BBF01D032D0DD
:106630008BC503F08A518BAF08D0000ED8808A55E5
:10664000006E000E8B55036E00500601F56F03C0FF
:10665000F6F6050108AF04D00601F6AF12D003D05C
:106660000601F6BF16D0050108510601F65D11E3DB
:1066700008E1F5510501075DD8A002D0060109D057
:10668000060105010A6B096B086B076B04011BD13E
:10669000060105018A510725016E8B51082101C0B1
:1066A00007F5086F0001A2EC2CF002C0F6F601C05D
:1066B000F5F6050108AF04D00601F6AF12D003D0FD
:1066C0000601F6BF15D0050108510601F65D10E37D
:1066D00008E1F5510501075DD8A002D0060108D0F8
:1066E000060105010A6B096B086B076B0401EBD00F
:1066F0000001A2EC2CF001500501075D006E025074
:10670000085900C007F5086F0601EC6BEB6BEC5302
:1067100030E1EB51B3082DE3D890EB35026EEC3548
:10672000036E0250F2CFF5F6F29CF29E03C0F7FF23
:1067300000016DEC04F00900F5CF03F00601F5BD92
:10674000F28CF5BFF28EF66F03C0F7F60501085123
:106750000601035C0AE308E1F6510501075DD8A0D4
:1067600002D0060102D0060104D0EB2BD8B4EC2BEA
:10677000CED7EB5308E1EC5306E105010A6B096B38
:106780000401A1D00601EB51D8B4EC07EB07ECC62D
:10679000F6F6EBC6F5F6F86B050EF76F000113EC95
:1067A00020F0320E060101240501096F000E0601DA
:1067B000022005010A6FD8900601EB35026EEC3518
:1067C000036E0250F2CFF5F6F29CF29E03C0F7FF83
:1067D00000016DEC04F00900F5CF03F00601F5BDF2
:1067E000F28CF5BFF28E0501075D0601ED6F0350D7
:1067F000050108590601EE6F010EEB25F56F000E3D
:10680000EC21F66FD890F535026EF635036E025026
:10681000F2CFF7F6F29CF29E03C0F7FF00016DEC99
:1068200004F00900F5CF03F00601F7BDF28CF7BFC5
:10683000F28EF86F03C0F9F6D890EB35026EEC35A6
:10684000036E0250F2CFFAF6F29CF29E03C0F7FFFD
:1068500000016DEC04F00900F5CF03F00601FABD6C
:10686000F28CFABFF28EF85DEF6F0350F959F06FBA
:10687000F0C6F6F6EFC6F5F6F86B050EF76F0001F9
:1068800006EC24F002C0F0F601C0EFF6EEC6F6F614
:10689000EDC6F5F6F0C6F8F6EFC6F7F606EC24F00E
:1068A00001500501092702500A230A5101080CE290
:1068B000FF0A03E10951BC0807E2030E0A6F090E43
:1068C000096F040100D0050100018FEF34F00501CC
:1068D0008E51000A000107E0010A0BE0030A1AE0EA
:1068E000010A1CE01FD005018E2B0001F8EF2EF0ED
:1068F0001DD005018E2B0401B7530BE1000159EFA8
:106900002FF00401B483640EB76F0001B6EF2FF0CF
:106910000DD0000150D405018E2B09D0BAD5050148
:106920008E2B05D005018E6B000100D00501000102
:10693000000C006A016A026A036A0601F96BFA6BCD
:10694000FB6BFC6BF851F711F611F5112CE0200EE2
:10695000FD6FD890F137F237F337F437F937FA375C
:10696000FB37FC37F851FC5D08E1F751FB5D05E1B1
:10697000F651FA5D02E1F551F95D0FE3F551F95F6A
:10698000F651D8A0F63DFA5FF751D8A0F73DFB5F6E
:10699000F851D8A0F83DFC5FD880003601360236A9
:1069A0000336FD2FD6D70000060EEA6EF90EE96E0B
:1069B0000001000CE9500601E96F3B0EF06F9A0EE2
:1069C000EF6FCA0EEE6FED6B0A0EEB6FE8C6F4F6D2
:1069D000E7C6F3F6E6C6F2F6E5C6F1F6F0C6F8F657
:1069E000EFC6F7F6EEC6F6F6EDC6F5F60001A1DF46
:1069F0000150EFCFE5F6ECCFE6F6ECCFE7F6ECCFC3
:106A0000E8F6005211E10601EB51010AD8A402D0C8
:106A100000010AD0E9510AE00F0BEB5D01E00CE246
:106A2000E9BD04D0200E03D00601E96B300E00262C
:106A300000509EA8FED7AD6EF0C6F4F6EFC6F3F692
:106A4000EEC6F2F6EDC6F1F6F86BF76BF66B0A0ED2
:106A5000F56F00016EDF03C0F0F602C0EFF601C073
:106A6000EEF600C0EDF60601EB2FB0D70001000CEA
:106A7000368036940A0E9EA8FED7AD6E0D0E9EA8E7
:106A8000FED7AD6E36B46AD0E3EC18F020DF040018
:106A90000501EB5357E10601D96BD951000145ECD3
:106AA00009F00601D92B006E00509EA8FED7AD6EEE
:106AB000070ED95DF2E1460EE96E06C5E8F605C59A
:106AC000E7F604C5E6F603C5E5F6000173DF0C0E34
:106AD0000601DA6FDA51000145EC09F00601DA2B04
:106AE000006E00509EA8FED7AD6E140EDA5DF2E186
:106AF000080EE96E08C5EDF607C5ECF60001FAECE4
:106B00001CF0190E0601DB6FDB51000145EC09F0AA
:106B10000601DB2B006E00509EA8FED7AD6E200E46
:106B2000DB5DF2E10A0EE96E0AC5EDF609C5ECF689
:106B30000001FAEC1CF00D0E9EA8FED7AD6E0A0EF9
:106B40000501EB6F81B008D00A0E9EA8FED7AD6E8E
:106B500081B002D00400FCD7000194D70A0E9EA891
:106B6000FED7AD6E0D0E9EA8FED7AD6E36905FEFD0
:106B700046F047EC0FF0DAC6DBF6DBC63FF4D9C6C9
:106B80003CF036B205D0E3EC18F0A1DE0400F9D7F2
:106B9000000C060E0601EB6FE60EEA6F440EEC6F7A
:106BA0000001B4EC28F0000CCBEC2CF002C0DAF6BB
:106BB00001C0D9F60601DB6BDB5100016BEC09F07B
:106BC0000601DB2B006E00509EA8FED7AD6E0D0EA9
:106BD000DB5DF2E1100EE96EDAC6EDF6D9C6ECF631
:106BE0000001FAEC1CF0200E9EA8FED7AD6E3A0E06
:106BF0009EA8FED7AD6E200E9EA8FED7AD6E070EE6
:106C00000601D96F020EDA6F0001B3DF3F5210E0C8
:106C10000601DE6B3F0EDD6F000124EC20F002C0A8
:106C2000DAF601C0D9F602C0E7F601C0E6F6B1DF38
:106C30000A0E9EA8FED7AD6E0D0E9EA8FED7AD6EB5
:106C400080EF46F0060E0601EB6FE80EEA6F460E87
:106C5000EC6F0001B4EC28F0000CA2EC2CF002C0A8
:106C6000DAF601C0D9F60601DB6BDB51000187ECD7
:106C700009F00601DB2B006E00509EA8FED7AD6E1A
:106C80000E0EDB5DF2E1100EE96EDAC6E5F6D9C64E
:106C9000E4F600012AEC24F0200E9EA8FED7AD6E8B
:106CA0003A0E9EA8FED7AD6E200E9EA8FED7AD6E02
:106CB000070E0601D96F020EDA6F00015ADF3F524C
:106CC00010E00601DE6B3F0EDD6F000124EC20F0CA
:106CD00002C0DAF601C0D9F602C0E9F601C0E8F652
:106CE000B1DF0A0E9EA8FED7AD6E0D0E9EA8FED790
:106CF000AD6EA1EF46F00601EB6BEB510001F5EC38
:106D000007F00601EB2B006E00509EA8FED7AD6E7B
:106D10001A0EEB5DF2E1100EE96EEAC6EDF6E9C679
:106D2000ECF60001FAEC1CF01D0E0601EC6FEC51C4
:106D30000001F5EC07F00601EC2B006E00509EA858
:106D4000FED7AD6E270EEC5DF2E1EB6BEB5100016F
:106D50001BEC08F00601EB2B006E00509EA8FED73E
:106D6000AD6E2B0EEB5DF2E1060EEC6F2E0E9EA8C3
:106D7000FED7AD6EEC2FFAD7356A346A355001086C
:106D80000BE303E13450F30807E30001E3EC18F0F0
:106D90009EDD04000601F2D7EB6BEB51000143ECE2
:106DA00008F00601EB2B006E00509EA8FED7AD6EDA
:106DB000060EEB5DF2E181B002D00400FCD7FA0EC2
:106DC000EB6F0001CCEC10F0000CE7C6F6F6E6C65F
:106DD000F5F60601F86B050EF76F000106EC24F0DE
:106DE00002C0E9F601C0E8F60A0E0601015CEA6F8E
:106DF000000E0258EB6FD890EA35026EEB35036E49
:106E00000250F2CFECF6F29CF29E03C0F7FF0001B5
:106E10006DEC04F00900F5CF03F00601ECBDF28C37
:106E2000ECBFF28E016E03C002F00001000C368050
:106E30000601E66BE65100016FEC08F00601E62B57
:106E4000006E00509EA8FED7AD6E2A0EE65DF2E100
:106E5000E56BE5510308D8A095D0D890E535036AD5
:106E6000F2CFE6F6F29CF29E000159EC08F0090020
:106E7000F5CF03F00601E6BDF28CE6BFF28EE76FB8
:106E800003C0E8F603C0EAF6E96F000134DFD890EA
:106E90000601E535036AF2CFE6F6F29CF29E0001A8
:106EA00059EC08F00900F5CF03F00601E6BDF28CBD
:106EB000E6BFF28EE76F03C0E8F6050EE75D006EF1
:106EC000000E0358036E00C001F005010A51035C77
:106ED00007E303E10150095D03E2060153D0050118
:106EE000D8900601E535036AF2CFE6F6F29CF29EF1
:106EF000000159EC08F00900F5CF03F00601E6BDEA
:106F0000F28CE6BFF28EE76F03C0E8F6050EE725C8
:106F1000016E000E0320036E035005010A5D06E3B7
:106F200003E10951015C02E206012CD00601E66B87
:106F3000E651000197EC08F00601E62B006E0050C8
:106F40009EA8FED7AD6E090EE65DF2E1100EE96E69
:106F50000AC5EDF609C5ECF60001FAEC1CF00C0EC2
:106F60000601E76FE751000197EC08F00601E72BF7
:106F7000006E00509EA8FED7AD6E220EE75DF2E1D6
:106F8000E52B67D7E55103081AE20A0E9EA8FED743
:106F9000AD6E0D0E9EA8FED7AD6EE66BE6510001FC
:106FA000BBEC08F00601E62B006E00509EA8FED751
:106FB000AD6E250EE65DF2E1010E016EF9D00A0E0E
:106FC0009EA8FED7AD6E0D0E9EA8FED7AD6EE66BE9
:106FD000E6510001E0EC08F00601E62B006E0050DF
:106FE0009EA8FED7AD6E090EE65DF2E1100EE96EC9
:106FF0000AC5EDF609C5ECF60001FAEC1CF00C0E22
:107000000601E76FE7510001E0EC08F00601E72B0D
:10701000006E00509EA8FED7AD6E310EE75DF2E126
:107020000A0E9EA8FED7AD6E0D0E9EA8FED7AD6EC1
:10703000E66BE65100010BEC09F00601E62B006E51
:1070400000509EA8FED7AD6E140EE65DF2E1020E72
:10705000EA6F1C0EE96F00014EDE06C5DCF605C5C1
:10706000DBF604C5DAF603C5D9F6010E0601EA6FB0
:10707000900EE96F00013FDE050103510601D95F63
:10708000050104510601DA5B050105510601DB5BD0
:10709000050106510601DC5B020EE76F1C0EE66F70
:1070A000000193DE0601E06BDF6B02C0DEF601C07B
:1070B000DDF6010EE76F900EE66F000186DE0150EF
:1070C0000601DD5F0250DE5B000EDF5BE05BDFC6CA
:1070D000E0F6DEC6DFF6DDC6DEF6DD6BE0C6F4F612
:1070E000DFC6F3F6DEC6F2F6DDC6F1F6DCC6F8F66C
:1070F000DBC6F7F6DAC6F6F6D9C6F5F6000119DCF6
:1071000003C0E0F602C0DFF601C0DEF600C0DDF627
:10711000DEC6E7F6DDC6E6F63CDD0A0E9EA8FED723
:10712000AD6E0D0E9EA8FED7AD6E0601E66BE65164
:10713000000128EC09F00601E62B006E00509EA825
:10714000FED7AD6E150EE65DF2E1E96BE86B00016E
:1071500079DD010E0601EA6FB80EE96F0001CBDDA3
:10716000010E0601E76FB80EE66F00012EDE01503A
:107170000501075D0601E16F02500501085906018E
:10718000E26FE36BE46BE2C6E7F6E1C6E6F6E2C661
:10719000E9F6E1C6E8F6000155DD0A0E9EA8FED725
:1071A000AD6E0D0E9EA8FED7AD6E000E016E0601EF
:1071B0000001000C0A0E9EA8FED7AD6E0D0E9EA813
:1071C000FED7AD6E369436B459D0E3EC18F067ECC8
:1071D00034F004000601D96BD9510001AFEC0BF07B
:1071E0000601D92B006E00509EA8FED7AD6E0A0E88
:1071F000D95DF2E1090EE96E8DC5E5F68CC5E4F6C0
:1072000000012AEC24F0040E0601DA6F200E9EA87D
:10721000FED7AD6EDA2FFAD70F0EDB6FDB51000110
:10722000AFEC0BF00601DB2B006E00509EA8FED7E2
:10723000AD6E1B0EDB5DF2E1490EE96E02C5E8F6AC
:1072400001C5E7F600C5E6F6FFC4E5F60001DAEC95
:1072500034F00D0E9EA8FED7AD6E81B00ED0BEEC00
:107260000FF00A0E9EA8FED7AD6E0D0E9EA8FED79B
:10727000AD6E81B002D00400FCD7A5D70A0E9EA83F
:10728000FED7AD6E0D0E9EA8FED7AD6EE5EF46F0B3
:107290003680010E0601EA6FC20EE96F00012BDD98
:1072A00006C5DCF605C5DBF604C5DAF603C5D9F676
:1072B000026A036A03C0E0F602C0DFF68DC5DEF69F
:1072C0008CC5DDF60601E36BE3510001D2EC0BF057
:1072D0000601E32B006E00509EA8FED7AD6E2C0E6B
:1072E000E35DF2E136B42DD00001E3EC18F067EC79
:1072F00034F004000601E36BE3510001FBEC0BF0FA
:107300000601E32B006E00509EA8FED7AD6E0A0E5C
:10731000E35DF2E1090EE96E8DC5E5F68CC5E4F694
:1073200000012AEC24F00D0E9EA8FED7AD6E81B0B0
:1073300006D0BEEC0FF081B002D00400FCD70601ED
:10734000D1D7010EEA6FC20EE96F0001D4DC05014E
:1073500003510601D95F050104510601DA5B0501FD
:1073600005510601DB5B050106510601DC5B8CC59E
:1073700000F08DC501F0026A036A01AE02D0020678
:107380000306DD51005EDE51015ADF51025AE05121
:10739000035A03C0E0F602C0DFF601C0DEF600C00B
:1073A000DDF6E46BD935E56FDA35E66FDB35E76F8F
:1073B000E537E637E737E537E637E737E537E637E6
:1073C000E737F00EE517E7C6F4F6E6C6F3F6E5C6CE
:1073D000F2F6E4C6F1F6E0C6F8F6DFC6F7F6DEC66A
:1073E000F6F6DDC6F5F6000199EC34F001C0E2F6E0
:1073F00000C0E1F60601E36BE351000116EC0CF06E
:107400000601E32B006E00509EA8FED7AD6E0A0E5B
:10741000E35DF2E1440EE96EE0C6E8F6DFC6E7F6AA
:10742000DEC6E6F6DDC6E5F60001DAEC34F00F0E56
:107430000601E46FE451000116EC0CF00601E42BA8
:10744000006E00509EA8FED7AD6E190EE45DF2E10D
:10745000460EE96EDCC6E8F6DBC6E7F6DAC6E6F607
:10746000D9C6E5F60001DAEC34F01E0E0601E56F30
:10747000E551000116EC0CF00601E52B006E005002
:107480009EA8FED7AD6E250EE55DF2E1040EE66F17
:10749000300E9EA8FED7AD6EE62FFAD7080EE96E25
:1074A000E2C6EDF6E1C6ECF60001FAEC1CF00D0EBA
:1074B0009EA8FED7AD6E06EF47F00A0E9EA8FED737
:1074C000AD6E0D0E9EA8FED7AD6E369436B44ED07E
:1074D000E3EC18F067EC34F004000501EB533AE1FB
:1074E0000601D96BD951000154EC0BF00601D92BE0
:1074F000006E00509EA8FED7AD6E060ED95DF2E17B
:107500000A0EE96E87C5E5F686C5E4F600012AECA9
:1075100024F00B0E0601DA6FDA51000154EC0BF087
:107520000601DA2B006E00509EA8FED7AD6E170E36
:10753000DA5DF2E10A0EE96E85C5E5F684C5E4F68A
:1075400000012AEC24F00D0E9EA8FED7AD6E0A0EA7
:107550000501EB6F81B008D00A0E9EA8FED7AD6E74
:1075600081B002D00400FCD70001B0D70A0E9EA85B
:10757000FED7AD6E0D0E9EA8FED7AD6E27EF47F07D
:10758000D2EC27F002C0DAF601C0D9F60601DB6BB7
:10759000DB51000175EC0BF00601DB2B006E005097
:1075A0009EA8FED7AD6E0F0EDB5DF2E1100EE96E08
:1075B000DAC6EDF6D9C6ECF60001FAEC1CF0200EA6
:1075C0009EA8FED7AD6E3A0E9EA8FED7AD6E200ED9
:1075D0009EA8FED7AD6E070E0601D96F020EDA6FB8
:1075E0000001B9EC35F03F5211E00601DE6B3F0EB1
:1075F000DD6F000124EC20F002C0DAF601C0D9F6FC
:1076000002C0E3F601C0E2F646EC29F00A0E9EA89D
:10761000FED7AD6E0D0E9EA8FED7AD6E48EF47F0BB
:10762000060E0601EB6FE20EEA6F400EEC6F0001F2
:10763000B4EC28F0000C79EC2CF002C0DAF601C0B2
:10764000D9F60601DB6BDB51000192EC0BF0060171
:10765000DB2B006E00509EA8FED7AD6E0E0EDB5DDC
:10766000F2E1100EE96EDAC6EDF6D9C6ECF60001CD
:10767000FAEC1CF0200E9EA8FED7AD6E3A0E9EA826
:10768000FED7AD6E200E9EA8FED7AD6E070E06018A
:10769000D96F020EDA6F0001B9EC35F03F5210E0FD
:1076A0000601DE6B3F0EDD6F000124EC20F002C00E
:1076B000DAF601C0D9F602C0E3F601C0E2F6B0DFA7
:1076C0000A0E9EA8FED7AD6E0D0E9EA8FED7AD6E1B
:1076D00069EF47F00601E76BE7510001A4EC09F000
:1076E0000601E72B006E00509EA8FED7AD6E1A0E65
:1076F000E75DF2E1100EE96EE6C6EDF6E5C6ECF6E2
:107700000001FAEC1CF01D0E0601E86FE8510001C3
:10771000A4EC09F00601E82B006E00509EA8FED7ED
:10772000AD6E350EE85DF2E10E0EE96F2E0E9EA8ED
:10773000FED7AD6EE92FFAD7356A346A35520BE1C0
:107740003450180808E30001E3EC18F067EC34F05B
:1077500004000601F3D7E76BE751000143EC08F0A2
:107760000601E72B006E00509EA8FED7AD6E060EF8
:10777000E75DF2E181B002D00400FCD7FA0EEB6FB6
:107780000001CCEC10F0000C36900601E26BE251E7
:107790000001E7EC09F00601E22B006E00509EA804
:1077A000FED7AD6E2F0EE25DF2E1030EE16F000138
:1077B000E3EC18F067EC34F0D8900601E135036A89
:1077C000F2CFE2F6F29CF29E0001D1EC09F0090042
:1077D000F5CF03F00601E2BDF28CE2BFF28EE36F5B
:1077E00003C0E4F603C0E6F6E56F000173DFD8904E
:1077F0000601E135036AF2CFE2F6F29CF29E000147
:10780000D1EC09F00900F5CF03F00601E2BDF28CDE
:10781000E2BFF28EE36F03C0E4F60A0EE325E56FE4
:10782000000E0320E66F0501875D0AE308E186513B
:107830000601E55DD8A002D0050102D005016FD098
:107840000A0E86250601E26F000E0501872106015A
:10785000E36FD890E135036AF2CFE4F6F29CF29E32
:107860000001D1EC09F00900F5CF03F00601E4BDF9
:10787000F28CE4BFF28E016EE351035C07E303E197
:107880000150E25D03E205014AD00601E26BE251DC
:10789000000111EC0AF00601E22B006E00509EA8D8
:1078A000FED7AD6E090EE25DF2E1100EE96E87C5FE
:1078B000EDF686C5ECF60001FAEC1CF00C0E0601A4
:1078C000E36FE351000111EC0AF00601E32B006EB7
:1078D00000509EA8FED7AD6E220EE35DF2E1E153AB
:1078E0001AE10A0E9EA8FED7AD6E0D0E9EA8FED719
:1078F000AD6EE26BE251000135EC0AF00601E22BBD
:10790000006E00509EA8FED7AD6E2B0EE25DF2E138
:10791000010E016E89D1E107040049D705010A0E65
:107920009EA8FED7AD6E0D0E9EA8FED7AD6E0601C9
:10793000E26BE25100015DEC0AF00601E22B006E01
:1079400000509EA8FED7AD6E090EE25DF2E1100E6A
:10795000E96E87C5EDF686C5ECF60001FAEC1CF081
:107960000C0E0601E36FE35100015DEC0AF0060125
:10797000E32B006E00509EA8FED7AD6E340EE35D83
:10798000F2E10A0E9EA8FED7AD6E0D0E9EA8FED7A0
:10799000AD6EE26BE25100018AEC0AF00601E22BC7
:1079A000006E00509EA8FED7AD6E240EE25DF2E19F
:1079B000050EE66FDC0EE56F00018CDE0601DC6B68
:1079C000DB6B85C5DAF684C5D9F6E66B320EE56F5A
:1079D000000180DE050184510601D95F0501855152
:1079E0000601DA5B000EDB5BDC5BE06BDF6B050E38
:1079F000DE6FAA0EDD6FDFC6E0F6DEC6DFF6DDC69F
:107A0000DEF6DD6BDE37DF37E037DE37DF37E037D6
:107A1000DE37DF37E037DE37DF37E037DE37DF37B7
:107A2000E037DE37DF37E037DE37DF37E037800E2D
:107A3000DE17E0C6F4F6DFC6F3F6DEC6F2F6DDC604
:107A4000F1F6DCC6F8F6DBC6F7F6DAC6F6F6D9C606
:107A5000F5F6000199EC34F003C0E0F602C0DFF661
:107A600001C0DEF600C0DDF6DEC6E3F6DDC6E2F6F6
:107A7000D7DD0A0E9EA8FED7AD6E0D0E9EA8FED7CE
:107A8000AD6E0601E26BE2510001AFEC0AF00601B7
:107A9000E22B006E00509EA8FED7AD6E260EE25D72
:107AA000F2E1E66BE56B000115DE0601E26BE251E7
:107AB0000001D5EC0AF00601E22B006E00509EA8F2
:107AC000FED7AD6E1E0EE25DF2E1100EE96E85C5C9
:107AD000EDF684C5ECF60001FAEC1CF0210E06016F
:107AE000E36FE3510001D5EC0AF00601E32B006ED1
:107AF00000509EA8FED7AD6E2E0EE35DF2E10501AB
:107B00008551010804E30DE18451B7080AE285516B
:107B10000108D8B077D0FF0A04E184513008D8B00A
:107B200071D00601E26BE2510001FFEC0AF00601A0
:107B3000E22B006E00509EA8FED7AD6E300EE25DC7
:107B4000F2E1E26BE25100012AEC0BF00601E22BBC
:107B5000006E00509EA8FED7AD6E2C0EE25DF2E1E5
:107B6000060EE36F2E0E9EA8FED7AD6EE32FFAD75A
:107B70000A0E9EA8FED7AD6E0A0E9EA8FED7AD6E69
:107B80000D0E9EA8FED7AD6EE26BE2510001AFEC88
:107B90000AF00601E22B006E00509EA8FED7AD6EE3
:107BA000260EE25DF2E1E66BE56B000193DD060176
:107BB000E26BE2510001D5EC0AF00601E22B006E07
:107BC00000509EA8FED7AD6E1E0EE25DF2E1100ED3
:107BD000E96E85C5EDF684C5ECF60001FAEC1CF003
:107BE000210E0601E36FE3510001D5EC0AF0060116
:107BF000E32B006E00509EA8FED7AD6E2E0EE35D07
:107C0000F2E17DD785C5E3F684C5E2F6000146ECD6
:107C100029F00A0E9EA8FED7AD6E0D0E9EA8FED7C7
:107C2000AD6E000E016E06010001000CA3EC24F005
:107C300002C0DAF601C0D9F60601DB6BDB510001A8
:107C400042EC0DF00601DB2B006E00509EA8FED723
:107C5000AD6E0C0EDB5DF2E1040EDC6F790E9EA8BA
:107C6000FED7AD6EDC2FFAD70C0EDD6FDD510001B3
:107C700042EC0DF00601DD2B006E00509EA8FED7F1
:107C8000AD6E140EDD5DF2E1DAC6EAFFD9C6E9FF9A
:107C9000000EEF1008E09EA8FED7EFCFADFFE92A57
:107CA000D8B4EA2AF5D7200E9EA8FED7AD6E3A0EBC
:107CB0009EA8FED7AD6E200E9EA8FED7AD6E080E14
:107CC000D96F020EDA6F0001B9EC35F03F5032087F
:107CD00011E00601D96BD951000161EC0DF00601EC
:107CE000D92B006E00509EA8FED7AD6E170ED95D41
:107CF000F2E112D00601EB6B3F0EEA6F4C0EEC6F17
:107D00000001B4EC28F00A0E9EA8FED7AD6E0D0E51
:107D10009EA8FED7AD6E06010001000C060E0601FE
:107D2000EB6FDB0EEA6F540EEC6F0001B4EC28F041
:107D3000C3EF3EF00601D96BD951000124EC0DF0E0
:107D40000601D92B006E00509EA8FED7AD6E170E0F
:107D5000D95DF2E1050ED96F020EDA6F0001B9ECC0
:107D600035F03F5210E00601DE6B3F0EDD6F000183
:107D700024EC20F002C0DAF601C0D9F602C0DCF62D
:107D800001C0DBF6CBD70A0E9EA8FED7AD6E0D0E56
:107D90009EA8FED7AD6E000C0A0E9EA8FED7AD6E53
:107DA0000D0E9EA8FED7AD6E369436B47FD0E3ECB0
:107DB00018F079EC12F004000601D96BD9510001DA
:107DC0003EEC0CF00601D92B006E00509EA8FED7A9
:107DD000AD6E070ED95DF2E12DC5E3F6030EE46F3B
:107DE000000172EC15F00B0E0601DA6FDA5100019A
:107DF0003EEC0CF00601DA2B006E00509EA8FED778
:107E0000AD6E0F0EDA5DF2E1080EE96E33C5EDF6E8
:107E100032C5ECF60001FAEC1CF0140E0601DB6F23
:107E2000DB5100013EEC0CF00601DB2B006E005034
:107E30009EA8FED7AD6E210EDB5DF2E156C5E3F6DE
:107E4000030EE46F000172EC15F0250E0601DC6FE5
:107E5000DC5100013EEC0CF00601DC2B006E005002
:107E60009EA8FED7AD6E290EDC5DF2E1080EE96E2C
:107E70005CC5EDF65BC5ECF60001FAEC1CF02E0ECD
:107E80000601DD6FDD5100013EEC0CF00601DD2B3B
:107E9000006E00509EA8FED7AD6E330EDD5DF2E1A0
:107EA000640EEB6F0001CCEC10F07FD70A0E9EA899
:107EB000FED7AD6E0D0E9EA8FED7AD6EEFEF47F06C
:107EC0000A0E9EA8FED7AD6E0D0E9EA8FED7AD6E13
:107ED000369436B49DD0E3EC18F067EC34F004002F
:107EE00006C5F4F605C5F3F604C5F2F603C5F1F6CA
:107EF0000601F86BF76B030EF66FE80EF56F0001E5
:107F000099EC34F003C0DCF602C0DBF601C0DAF60F
:107F100000C0D9F60601DD6BDD5100013EEC0CF02E
:107F20000601DD2B006E00509EA8FED7AD6E070E39
:107F3000DD5DF2E1FEC4E3F6030EE46F000172ECD6
:107F400015F00B0E0601DE6FDE5100013EEC0CF069
:107F50000601DE2B006E00509EA8FED7AD6E0F0E00
:107F6000DE5DF2E1450EE96EDCC6E8F6DBC6E7F65B
:107F7000DAC6E6F6D9C6E5F60001DAEC34F0140EFE
:107F80000601DF6FDF5100013EEC0CF00601DF2B34
:107F9000006E00509EA8FED7AD6E210EDF5DF2E1AF
:107FA0007FC5E3F6030EE46F000172EC15F0250EB9
:107FB0000601E06FE05100013EEC0CF00601E02B01
:107FC000006E00509EA8FED7AD6E290EE05DF2E176
:107FD000080EE96E85C5EDF684C5ECF60001FAECF5
:107FE0001CF02E0E0601E16FE15100013EEC0CF099
:107FF0000601E12B006E00509EA8FED7AD6E330E39
:10800000E15DF2E1640EEB6F0001CCEC10F061D7A2
:108010000A0E9EA8FED7AD6E0D0E9EA8FED7AD6EC1
:1080200010EF48F00601D96BD9510001A8EC0CF013
:108030000601D92B006E00509EA8FED7AD6E2C0E07
:10804000D95DF2E1369436B43DD00001E3EC18F08E
:1080500067EC34F087868788FA0E0601EB6F000123
:10806000CCEC10F0FA0E0601EB6F0001CCEC10F036
:10807000FA0E0601EB6F0001CCEC10F0FA0E0601CF
:10808000EB6F0001CCEC10F0040087968798FA0E95
:108090000601EB6F0001CCEC10F0FA0E0601EB6F5D
:1080A0000001CCEC10F0FA0E0601EB6F0001CCECF5
:1080B00010F0FA0E0601EB6F0001CCEC10F004009A
:1080C0000601C1D70A0E9EA8FED7AD6E0D0E9EA862
:1080D000FED7AD6E000131EF48F00601E46BE36BB3
:1080E0000001C9EC26F00601D96BD9510408D8A0CB
:1080F0006ED0DC6BDC51000157EC03F00601DC2B89
:10810000006E00509EA8FED7AD6E090EDC5DF2E158
:10811000D9C6E3F61B0EE46F000172EC15F00B0EEE
:108120000601DD6FDD51000157EC03F00601DD2B88
:10813000006E00509EA8FED7AD6E0F0EDD5DF2E121
:10814000DA6BDA511F0841E3DC6BDC51000171ECA2
:1081500003F00601DC2B006E00509EA8FED7AD6E2A
:10816000040EDC5DF2E1DAC6E3F6010EE46F000115
:1081700072EC15F0200E9EA8FED7AD6E3A0E9EA8AA
:10818000FED7AD6E0601DB6BDB510F081CE300016F
:1081900022EC27F001C0DCF6200E9EA8FED7AD6EC3
:1081A000300E9EA8FED7AD6E780E9EA8FED7AD6E9F
:1081B000DCC6EDF6570E0601EE6F000139EC15F046
:1081C0000601DB2BE1D7DA2BBCD7D92B8ED70A0ED1
:1081D0009EA8FED7AD6E0D0E9EA8FED7AD6E000117
:1081E00052EF48F0040152C401F0000137EF41F0B2
:1081F00004019BC401F09CC402F00001000C0601C4
:10820000DF6BE06B00018CEC26F018EC21F0012C08
:108210002DD00601D9530FE0E16BE151000122ECB2
:1082200002F00601E12B006E00509EA8FED7AD6E55
:108230000E0EE15DF2E10001BEEC13F0015216E01A
:108240000601D9530FE0E16BE15100013CEC02F073
:108250000601E12B006E00509EA8FED7AD6E400EC9
:10826000E15DF2E1FE0E016E9FD10001BBD7012C52
:1082700013D00601D9530FE0E16BE15100016FEC1F
:1082800002F00601E12B006E00509EA8FED7AD6EF5
:108290000D0EE15DF2E10001D6CFDCF60601D95109
:1082A00001081FE2E16BE151000188EC02F00601D8
:1082B000E12B006E00509EA8FED7AD6E0B0EE15D67
:1082C000F2E1DCC6E3F61B0EE46F000172EC15F080
:1082D0000A0E9EA8FED7AD6E0D0E9EA8FED7AD6EFF
:1082E0000601D9530FE0E16BE1510001A2EC02F06D
:1082F0000601E12B006E00509EA8FED7AD6E070E62
:10830000E15DF2E1DCC6DBF6DE6BDD6BDE517F08A2
:108310001AE303E1DD51BF0816E30400DB51DB2B58
:10832000E16FE26FE36B0001DDEC21F00601DB534E
:1083300006E1D95304E02E0E9EA8FED7AD6EDD2BCC
:10834000D8B4DE2BE3D7E26B010EE36F0001DDEC66
:1083500021F00601D9530FE0E16BE1510001B8ECC7
:1083600002F00601E12B006E00509EA8FED7AD6E14
:10837000090EE15DF2E1E46BE36B0001C9EC26F06C
:10838000DCC6DBF60601DE6BDD6BDE517F08D8A0B4
:10839000B4D004E1DD51BF08D8A0AFD00400000183
:1083A00022EC27F001C0DAF60601DB51DA5DD8B421
:1083B00097D0DF2BD8B4E02BD9510108D8B08FD09B
:1083C000000116DF02C0E2F601C0E1F6010E06016F
:1083D000015CE36F000E0258E46F000109DF02C088
:1083E000E6F601C0E5F6010E0601015CE76F000E3E
:1083F0000258E86FE96BE9510001CFEC02F0060189
:10840000E92B006E00509EA8FED7AD6E050EE95D0B
:10841000F2E1DAC6EDF6570EEE6F000139EC15F019
:10842000070E0601EA6FEA510001CFEC02F00601E7
:10843000EA2B006E00509EA8FED7AD6E130EEA5DCB
:10844000F2E1DBC6EDF6570EEE6F000139EC15F0E8
:10845000150E0601EB6FEB510001CFEC02F00601A7
:10846000EB2B006E00509EA8FED7AD6E190EEB5D93
:10847000F2E1100EE96EE4C6EDF6E3C6ECF600019B
:10848000FAEC1CF01C0E0601EC6FEC510001CFEC75
:1084900002F00601EC2B006E00509EA8FED7AD6ED8
:1084A000200EEC5DF2E1E8C6EDF6570EEE6F00012E
:1084B00039EC15F0E7C6EDF6570E0601EE6F000138
:1084C00039EC15F0290E9EA8FED7AD6E0A0E9EA8B7
:1084D000FED7AD6E0D0E9EA8FED7AD6E060108D07C
:1084E000DB5306E1D95304E02E0E9EA8FED7AD6EF5
:1084F000DB2BDD2BD8B4DE2B48D7D951010829E27C
:10850000E16BE1510001F5EC02F00601E12B006E98
:1085100000509EA8FED7AD6E1B0EE15DF2E1100E7D
:10852000E96EE0C6EDF6DFC6ECF60001FAEC1CF0F1
:108530001E0E0601E26FE2510001F5EC02F00601A9
:10854000E22B006E00509EA8FED7AD6E2A0EE25DB3
:10855000F2E1DF5302E1E05314E0D92D0FD0E16BDB
:10856000E15100011DEC03F00601E12B006E00500B
:108570009EA8FED7AD6E250EE15DF2E1FF0E016E05
:1085800013D0D92D0FD0E16BE151000142EC03F083
:108590000601E12B006E00509EA8FED7AD6E040EC2
:1085A000E15DF2E1000E016E0001000C0601DA51FE
:1085B000DC19800BDE6FDAAF05D0D91FDA1FD92B9B
:1085C000D8B4DA2BDCAF05D0DB1FDC1FDB2BD8B433
:1085D000DC2B016A026A006A036ADC5102E1DB51AA
:1085E00018E0100EDD6FD890D937DA370036033631
:1085F000DC51035C02E1DB51005C07E3DB51005E10
:10860000D8A00306DC51035ED88001360236DD2F88
:10861000EAD70000DEAF05D0011E021E012AD8B441
:10862000022A00012EEF43F00A0E9EA8FED7AD6E7F
:108630000D0E9EA8FED7AD6E369436B441D0E3EC55
:1086400018F067EC34F004008DC5DAF68CC5D9F665
:108650000601DC6B640EDB6F0001A8D702C0DAF6FE
:1086600001C0D9F60601DB6BDB510001D1EC0CF047
:108670000601DB2B006E00509EA8FED7AD6E1E0ECD
:10868000DB5DF2E10C0EE96EDAC6E5F6D9C6E4F67A
:1086900000012AEC24F0430E9EA8FED7AD6E200EFA
:1086A0009EA8FED7AD6E0D0E9EA8FED7AD6E81B012
:1086B00006D0BEEC0FF081B002D00400FCD7BDD7CD
:1086C0000A0E9EA8FED7AD6E0D0E9EA8FED7AD6E0B
:1086D00098EF48F00601DB6BDA511F080FE3040046
:1086E0000001E3EC18F079EC12F005012D510601C0
:1086F000DB5D03E0DA2B2DC5DBF6EED7D95101089F
:1087000043E2DC6BDC5100016AEC0CF00601DC2B6F
:10871000006E00509EA8FED7AD6E0B0EDC5DF2E140
:10872000080EE96E33C5EDF632C5ECF60001FAEC41
:108730001CF0100E0601DD6FDD5100016AEC0CF03B
:108740000601DD2B006E00509EA8FED7AD6E1F0EF9
:10875000DD5DF2E1080EE96E5CC5EDF65BC5ECF699
:108760000001FAEC1CF0240E0601DE6FDE51000160
:108770006AEC0CF00601DE2B006E00509EA8FED7BE
:10878000AD6E290EDE5DF2E105013351110822E2E2
:10879000FF0A03E13251F2081DE25C5111081AE2AE
:1087A000FF0A03E15B51F20815E20601D92D0FD053
:1087B000DC6BDC51000142EC03F00601DC2B006EA7
:1087C00000509EA8FED7AD6E040EDC5DF2E1000EF7
:1087D000016E14D00601D92D0FD0DC6BDC510001E5
:1087E00091EC0CF00601DC2B006E00509EA8FED729
:1087F000AD6E080EDC5DF2E1FF0E016E0001000CB3
:108800000A0E9EA8FED7AD6E0D0E9EA8FED7AD6EC9
:10881000369436B45AD0E3EC18F067EC34F0040028
:1088200005018F5164081EE10601D96BD951000181
:10883000F7EC0CF00601D92B006E00509EA8FED775
:10884000AD6E040ED95DF2E1060EDA6F200E9EA821
:10885000FED7AD6EDA2FFAD70D0E9EA8FED7AD6EFD
:1088600032D005018F5132081BE14C0E9EA8FED775
:10887000AD6E4F0E9EA8FED7AD6E570E9EA8FED7CA
:10888000AD6E070E0601D96F200E9EA8FED7AD6E05
:10889000D92FFAD70D0E9EA8FED7AD6E14D00501C4
:1088A0008F51140810E10601D96BD95100010CEC6D
:1088B0000DF00601D92B006E00509EA8FED7AD6EBC
:1088C0000B0ED95DF2E10001A4D70A0E9EA8FED7D7
:1088D000AD6E0D0E9EA8FED7AD6EDEEF48F0020E17
:1088E0000601D96F0001B1EC15F001BE06D0020EF1
:1088F0000601D96F000136EC17F0FFEF48F0060EC5
:108900000601EB6FD90EEA6F480EEC6F0001B4EC74
:1089100028F03BEF45F0060E0601EB6FD90EEA6F2B
:10892000490EEC6F0001B4EC28F040EF45F0060E64
:108930000601EB6FD90EEA6F4B0EEC6F0001B4EC41
:1089400028F0F2CFDAF6F29CF29EAA6A4B0EA96EDC
:10895000A69CA69EA680A8500601DABDF28CDABFBE
:10896000F28E0401436F000144EF45F00601D96B1C
:10897000D951000142EC06F00601D92B006E0050DF
:108980009EA8FED7AD6E180ED95DF2E1010ED96F2B
:10899000000135DC01BE01D001D0B8D00601D96B91
:1089A000D951000161EC06F00601D92B006E005090
:1089B0009EA8FED7AD6E230ED95DF2E1040EDA6FEC
:1089C0002E0E9EA8FED7AD6EDA2FFAD7010ED96F04
:1089D000000180DE01BE01D012D00601D96BD95151
:1089E000000185EC06F00601D92B006E00509EA810
:1089F000FED7AD6E2A0ED95DF2E1000187D017ECEB
:108A000037F00152FCE0C4EC3BF00152FCE00601FF
:108A1000D96BD9510001ADEC06F00601D92B006EDF
:108A200000509EA8FED7AD6E180ED95DF2E1000190
:108A300016EC3EF0D3EC1CF002C0DAF601C0D9F619
:108A40000601013C15D0DA3D13D0D96BD951000194
:108A5000CCEC06F00601D92B006E00509EA8FED784
:108A6000AD6E1B0ED95DF2E100019AEC3EF00601FD
:108A7000D96B000144D70601DA6BD96B00014BD7E3
:108A80000601D96B000153D7010E0601D96F000111
:108A9000B1EC15F001AE01D039D0010E0601D96F4D
:108AA000000136EC17F0F4EC2CF00A0E9EA8FED76D
:108AB000AD6E0D0E9EA8FED7AD6E030E0601D96FEA
:108AC0002D0E9EA8FED7AD6ED92FFAD7020EDA6F03
:108AD000DA510001ECEC06F00601DA2B006E0050D2
:108AE0009EA8FED7AD6E160EDA5DF2E1030EDB6FC7
:108AF0002D0E9EA8FED7AD6EDB2FFAD70A0E9EA8CC
:108B0000FED7AD6E0D0E9EA8FED7AD6E00016AEFCA
:108B100049F0050E0601DA6FEC0ED96F0001ACECDE
:108B20001FF002C0DAF601C0D9F60601DC6B3F0E79
:108B3000DB6F050EDE6FEC0EDD6F01C0DFF60001AE
:108B4000CAEC1FF001520FE10501935306E1030E39
:108B50000601D96F0001A1EC11F00401B485000EEB
:108B6000016E72EF49F0060E0601DA6FD30ED96F6F
:108B70000001ACEC1FF002C0DAF601C0D9F6060124
:108B8000DC6B3F0EDB6F060EDE6FD30EDD6F01C0B8
:108B9000DFF60001CAEC1FF0015206E16BEC2CF08D
:108BA000000E016E04019ED3060E0601DA6F010E5F
:108BB000D96F0001ACEC1FF002C0DAF601C0D9F6A3
:108BC0000601DC6B3F0EDB6F060EDE6F010EDD6F04
:108BD00001C0DFF60001CAEC1FF0015206E1F4EC1F
:108BE0002CF0000E016E04017DD3050E0601DA6F34
:108BF000FA0ED96F0001ACEC1FF002C0DAF601C02A
:108C0000D9F60601DC6B3F0EDB6F050EDE6FFA0E48
:108C1000DD6F01C0DFF60001CAEC1FF0015232E146
:108C20000601D96BD951000104EC06F00601D92BDD
:108C3000006E00509EA8FED7AD6E090ED95DF2E120
:108C4000DA6BDA510001ABEC05F0000906E0060131
:108C5000DA2B9EA8FED7AD6EF4D70B0E0601DB6FA4
:108C6000DB51000104EC06F00601DB2B006E005026
:108C70009EA8FED7AD6E0F0EDB5DF2E1000E016E19
:108C8000040130D3060E0601DA6F230ED96F0001FE
:108C9000ACEC1FF002C0DAF601C0D9F60601DC6BBD
:108CA0003F0EDB6F060EDE6F230EDD6F01C0DFF6B9
:108CB0000001CAEC1FF0015206E138EF35F0000E5A
:108CC000016E04010FD3060E0601DA6F2B0ED96F69
:108CD0000001ACEC1FF002C0DAF601C0D9F60601C3
:108CE000DC6B3F0EDB6F060EDE6F2B0EDD6F01C0FF
:108CF000DFF60001CAEC1FF0015206E1D4EF35F0B7
:108D0000000E016E0401EED2060E0601DA6F340E7B
:108D1000D96F0001ACEC1FF002C0DAF601C0D9F641
:108D20000601DC6B3F0EDB6F060EDE6F340EDD6F6F
:108D300001C0DFF60001CAEC1FF0015206E12DEF81
:108D400036F0000E016E0401CDD2060E0601DA6F78
:108D50003E0ED96F0001ACEC1FF002C0DAF601C084
:108D6000D9F60601DC6B3F0EDB6F060EDE6F3E0EA2
:108D7000DD6F01C0DFF60001CAEC1FF0015208E10F
:108D800017EC37F00152FCE0000E016E0401AAD28C
:108D9000060E0601DA6F6B0ED96F0001ACEC1FF006
:108DA00002C0DAF601C0D9F60601DC6B3F0EDB6FBC
:108DB000060EDE6F6B0EDD6F01C0DFF60001CAEC40
:108DC0001FF0015206E1DAEF38F0000E016E0401E7
:108DD00089D2060E0601DA6F730ED96F0001ACEC72
:108DE0001FF002C0DAF601C0D9F60601DC6B3F0EB7
:108DF000DB6F060EDE6F730EDD6F01C0DFF6000164
:108E0000CAEC1FF0015206E148EF39F0000E016E86
:108E1000040168D2060E0601DA6F450ED96F000113
:108E2000ACEC1FF002C0DAF601C0D9F60601DC6B2B
:108E30003F0EDB6F060EDE6F450EDD6F01C0DFF605
:108E40000001CAEC1FF0015206E15DEF3AF0000E9E
:108E5000016E040147D2060E0601DA6F580ED96F73
:108E60000001ACEC1FF002C0DAF601C0D9F6060131
:108E7000DC6B3F0EDB6F060EDE6F580EDD6F01C040
:108E8000DFF60001CAEC1FF0015206E1C0EF3AF034
:108E9000000E016E040126D2060E0601DA6F4E0E98
:108EA000D96F0001ACEC1FF002C0DAF601C0D9F6B0
:108EB0000601DC6B3F0EDB6F060EDE6F4E0EDD6FC4
:108EC00001C0DFF60001CAEC1FF0015206E11BEF02
:108ED0003BF0000E016E040105D2060E0601DA6FAA
:108EE000630ED96F0001ACEC1FF002C0DAF601C0CE
:108EF000D9F60601DC6B3F0EDB6F060EDE6F630EEC
:108F0000DD6F01C0DFF60001CAEC1FF0015208E17D
:108F1000C4EC3BF00152FCE0000E016E0401E2D112
:108F2000060E0601DA6F0A0ED96F0001ACEC1FF0D5
:108F300002C0DAF601C0D9F60601DC6B3F0EDB6F2A
:108F4000060EDE6F0A0EDD6F01C0DFF60001CAEC0F
:108F50001FF0015206E116EC3EF0000E016E040116
:108F6000C1D1060E0601DA6F160ED96F0001ACEC06
:108F70001FF002C0DAF601C0D9F60601DC6B3F0E25
:108F8000DB6F060EDE6F160EDD6F01C0DFF600012F
:108F9000CAEC1FF0015206E19AEC3EF0000E016EA1
:108FA0000401A0D1060E0601DA6F910ED96F0001FF
:108FB000ACEC1FF002C0DAF601C0D9F60601DC6B9A
:108FC0003F0EDB6F060EDE6F910EDD6F01C0DFF628
:108FD0000001CAEC1FF0015206E1CCEF3EF0000E9A
:108FE000016E04017FD1060E0601DA6F9A0ED96F69
:108FF0000001ACEC1FF002C0DAF601C0D9F60601A0
:10900000DC6B3F0EDB6F060EDE6F9A0EDD6F01C06C
:10901000DFF60001CAEC1FF0015206E160EF3FF0FD
:10902000000E016E04015ED1060E0601DA6FA30E7A
:10903000D96F0001ACEC1FF002C0DAF601C0D9F61E
:109040000601DC6B3F0EDB6F060EDE6FA30EDD6FDD
:1090500001C0DFF60001CAEC1FF0015206E112EF79
:1090600040F0000E016E04013DD1060E0601DA6FDC
:10907000850ED96F0001ACEC1FF002C0DAF601C01A
:10908000D9F60601DC6B3F0EDB6F060EDE6F850E38
:10909000DD6F01C0DFF60001CAEC1FF0015206E1EE
:1090A0006DEF40F0000E016E04011CD1060E0601AA
:1090B000DA6F7A0ED96F0001ACEC1FF002C0DAF65D
:1090C00001C0D9F60601DC6B3F0EDB6F060EDE6FCA
:1090D0007A0EDD6F01C0DFF60001CAEC1FF001520D
:1090E0000AE1FF0E0601D96F0001FFEC40F0000E0F
:1090F000016E0401F7D0060E0601DA6FAF0ED96FCC
:109100000001ACEC1FF002C0DAF601C0D9F606018E
:10911000DC6B3F0EDB6F060EDE6FAF0EDD6F01C046
:10912000DFF60001CAEC1FF0015206E114EF43F034
:10913000000E016E0401D6D0060E0601DA6FC30ED2
:10914000D96F0001ACEC1FF002C0DAF601C0D9F60D
:109150000601DC6B3F0EDB6F060EDE6FC30EDD6FAC
:1091600001C0DFF60001CAEC1FF001520AE1FF0E58
:109170000601D96F00016AEC43F0000E016E040194
:10918000B1D0060E0601DA6FB90ED96F0001ACEC52
:109190001FF002C0DAF601C0D9F60601DC6B3F0E03
:1091A000DB6F060EDE6FB90EDD6F01C0DFF600016A
:1091B000CAEC1FF0015206E100EF44F0000E016E10
:1091C000040190D0060E0601DA6FCC0ED96F0001B3
:1091D000ACEC1FF002C0DAF601C0D9F60601DC6B78
:1091E0003F0EDB6F060EDE6FCC0EDD6F01C0DFF6CB
:1091F0000001CAEC1FF0015206E16FEF44F0000ECF
:10920000016E04016FD0050E0601DA6FF30ED96FFF
:109210000001ACEC1FF002C0DAF601C0D9F606017D
:10922000DC6B3F0EDB6F050EDE6FF30EDD6F01C0F2
:10923000DFF60001CAEC1FF001522FE10601D96BE5
:10924000D95100011EEC06F00601D92B006E00502A
:109250009EA8FED7AD6E200ED95DF2E1030EDA6F47
:109260002E0E9EA8FED7AD6EDA2FFAD70A0E9EA854
:10927000FED7AD6E0D0E9EA8FED7AD6E000147EC79
:109280000FF00601DB6BDBC63FF4D96B0001A1ECEC
:1092900011F0000E016E040125D0050E0601DA6FF3
:1092A000FE0ED96F0001ACEC1FF002C0DAF601C06F
:1092B000D9F60601DC6B3F0EDB6F050EDE6FFE0E8E
:1092C000DD6F01C0DFF60001CAEC1FF0015207E1BB
:1092D000B6EF44F0000E016E040104D00001FF0E51
:1092E000016E04010001000C0401415302E14253EC
:1092F0000DE032520BE1335209E19D9A878E000155
:1093000069EC0FF09D8A879E19D0040136B203D014
:10931000000114D00401516B506B0A0E386E00012D
:1093200076EF1FF001BE01D007D060EF2AF001BE3A
:1093300001D002D089EC45F047EC0FF0000C305220
:1093400002E1315201E00FD0316A640E306E040147
:10935000502BD8B4512B515303E15051770804E2FC
:1093600000016BEC2CF00401050157EF4BF077EC9A
:1093700027F002C0D9F601C0D8F6060102507E08D7
:1093800008E2FF0A03E1D851BF0803E2010E016EB3
:1093900002D0000E016E0001D9EF49F00501925391
:1093A00001E058D09C2BD8B49D2B140E926F000175
:1093B000DED7015204E005EC23F005014BD0050196
:1093C0009D51D1080AE2FF0A03E19C51EF0805E232
:1093D000000105EC23F005013DD0030E8625016E4A
:1093E000000E8721036E0350A15D04E318E1A05134
:1093F000015C15E3030EA0250601D86F000E0501E0
:10940000A1210601D96F0501875D24E308E186519A
:109410000601D85DD8A002D005011CD005019DC56C
:10942000D9F69CC5D8F6A1C5DBF6A0C5DAF60601CB
:10943000DC6B00018AEC22F09DC5D9F69CC5D8F6FC
:1094400087C5DBF686C5DAF60601DC6B00018AEC1F
:1094500022F00501000107EF4BF036AA03D0010E00
:10946000016E02D0000E016E13EF4BF036B203D046
:10947000000E016E3AD089EC45F001C0D8F6060125
:10948000D8AF0FD0D96BD9510001D5EC05F006014A
:10949000D92B006E00509EA8FED7AD6E0F0ED95D81
:1094A000F2E105019351040804E0D8C601F000017F
:1094B0001CD00601D96BD9510001EFEC05F0060173
:1094C000D92B006E00509EA8FED7AD6E040ED95D5C
:1094D000F2E1000147EC0FF0010E0601DB6FDBC685
:1094E0003FF43C0E3C6ED8C601F0050157EF4BF03F
:1094F00005019351F60FD8B0DAD00A0F00015AEFE8
:109500004BF079EC12F005013351100814E2FF0A18
:1095100003E1325194080FE25C5110080CE2FF0A9B
:1095200003E15B51940807E2080E0601D96F0001C0
:10953000A1EC11F00501BBD01BEF15F0015206E1C3
:10954000070E0601D96F0001A1EC11F00501AFD0A3
:1095500081A406D0060E0601D96F0001A1EC11F01E
:109560000501A5D0CEEF18F0050E0601D96F000158
:10957000A1EC11F005019BD096EF1DF0E3EC18F083
:1095800008EF1EF001520EE036B607D0030E0601BA
:10959000D96F0001A1EC11F005D00601D96B0001D3
:1095A000A1EC11F0050183D00501855111080DE2F0
:1095B000FF0A03E184515C0808E2030E0601D96F3B
:1095C0000001A1EC11F072D00501355203E13450D5
:1095D0000A0806E236800401516B506B04D0050185
:1095E00036908796879800017FDEE3EC18F067ECF1
:1095F00034F0A5D63550000808E2FF0A03E13450E4
:109600002C0803E205EC23F051D06EDEC7D6E3EC64
:1096100018F067EC34F005014AD0E3EC18F067EC81
:1096200034F062DE1AD7015203E1050140D0000197
:10963000355207E134500A0804E30401B4A52FD0E1
:1096400000010601D86BD85100017FEC0DF0060136
:10965000D82B006E00509EA8FED7AD6E1C0ED85DB4
:10966000F2E1D86BD8510001EFEC05F00601D82BE0
:10967000006E00509EA8FED7AD6E040ED85DF2E1DC
:10968000000147EC0FF0010E0601DB6FDBC63FF473
:109690003C0E3C6E040ED96F0001A1EC11F00501E7
:1096A00006D0E3EC18F067EC34F0E0D605010001D9
:1096B00087EF4EF0F2CF0EF0F29CF29EE824E50F19
:1096C000F66E960EF76ED8B0F72A000EF86EFB6EA7
:1096D0000A00F550FA6E0800F5500EBCF28C0EBE72
:1096E000F28EF96EA895F495AC961A96A296789596
:1096F0006495509538950295F86AF1849F9AD08EBA
:109700000D8EEA6AE96AC150C00B0F09C16E070EDF
:10971000B46EB450A19C500EAF6E260EAC6E900E7F
:10972000AB6E2A6A2B6A010E2C6E2D6A2E6A2F6A86
:10973000306A316A326A336A346A356A3690376A17
:10974000386A396A3A6A3B6A3C6A36923D6A3E6ACE
:1097500004013F6B406B416B426B36943696446B11
:10976000456B466B476B486B496B4A6B4B6B4C6B5D
:10977000506B516B526BFF0E536F546B556F566BA2
:10978000576B586B596B5A6BB06B3698369AB26BF5
:10979000B36B369C369EB491B493B56BB66BB76B16
:1097A000B86BB96BBA6BBB6BBC6BBD6BFE6BFF6B05
:1097B0000501006B016B026B036B046B056B066BA1
:1097C000076B086B096B0A6B2D6B2E6B2F6B306B65
:1097D000316B326B336B566B576B586B596B5A6BE3
:1097E0005B6B5C6B5D6B5E6B7F6B806B816B826BAD
:1097F000836B846B856B866B876B886B896B8A6BDD
:109800008B6B8C6B8D6B8E6B640E8F6F906B916B13
:10981000926B946B956B966B976B986B996B9A6B3D
:109820009B6B9C6B9D6B9E6B9F6BA06BA16BA26BEC
:10983000A36B570EA46F700EA56F300EA66F310E7E
:10984000A76FA86B570EA96F700EAA6F300EAB6F83
:10985000320EAC6F3A0EAD6FAE6B570EAF6F700E2F
:10986000B06F320EB16F520EB26FB36B570EB46F52
:10987000700EB56F300EB66F330EB76F3A0EB86F0D
:10988000B96B570EBA6F700EBB6F330EBC6F520EB2
:10989000BD6FBE6B570EBF6F700EC06F300EC16FC5
:1098A000340EC26F3A0EC36FC46B570EC56F700E85
:1098B000C66F340EC76F520EC86FC96B570ECA6F92
:1098C000700ECB6F300ECC6F350ECD6FCE6B570E4A
:1098D000CF6F700ED06F300ED16F360ED26FD36B4C
:1098E000570ED46F700ED56F310ED66FD76FD86B01
:1098F000570ED96F700EDA6F310EDB6F320EDC6FE0
:10990000DD6B570EDE6F700EDF6F310EE06F330EC2
:10991000E16F430EE26F4C0EE36F520EE46FE56BA6
:10992000570EE66F700EE76F310EE86F340EE96F79
:10993000EA6BEB6B0401B495430E0501EC6F410E2D
:10994000ED6F4C0EEE6F490EEF6F420EF06F310E61
:10995000F16FF26B530EF36F570EF46F490EF56F04
:10996000540EF66F430EF76F480EF86FF96B560EF4
:10997000FA6F450EFB6F520EFC6FFD6B470EFE6FCC
:109980004F0EFF6F0601006B430E016F410E026F19
:109990004C0E036F200E046F530E056F480E066FBA
:1099A0004F0E076F570E086F096B530E0A6F450E67
:1099B0000B6F540E0C6F200E0D6F430E0E6F410E89
:1099C0000F6F4C0E106F440E116F410E126F540E3C
:1099D000136F450E146F156B500E166F520E176FE6
:1099E0004F0E186F420E196F450E1A6F200E1B6F27
:1099F000530E1C6F450E1D6F520E1E6F490E1F6FCA
:109A0000410E206F4C0E216F226B490E236F520EB8
:109A1000246F200E256F530E266F480E276F4F0EB2
:109A2000286F570E296F2A6B490E2B6F520E2C6F21
:109A3000200E2D6F530E2E6F430E2F6F410E306F81
:109A40004C0E316F450E326F336B490E346F520E30
:109A5000356F200E366F4F0E376F460E386F396FE9
:109A6000530E3A6F450E3B6F540E3C6F3D6B490EE3
:109A70003E6F520E3F6F200E406F430E416F410EFE
:109A8000426F4C0E436F446B500E456F530E466F42
:109A9000490E476F200E486F530E496F480E4A6FAC
:109AA0004F0E4B6F570E4C6F4D6B500E4E6F530E4B
:109AB0004F6F490E506F200E516F530E526F430E71
:109AC000536F410E546F4C0E556F450E566F576BCA
:109AD000500E586F530E596F490E5A6F200E5B6F20
:109AE0004F0E5C6F460E5D6F5E6F530E5F6F450EDF
:109AF000606F540E616F626B500E636F530E646F34
:109B0000490E656F200E666F430E676F410E686FDA
:109B10004C0E696F6A6B430E6B6F4A0E6C6F200EB2
:109B20006D6F530E6E6F480E6F6F4F0E706F570E46
:109B3000716F726B430E736F4A0E746F200E756FE8
:109B4000430E766F410E776F4C0E786F796B540E23
:109B50007A6F450E7B6F530E7C6F540E7D6F200E17
:109B60007E6F460E7F6F4C0E806F410E816F530EDD
:109B7000826F480E836F846B500E856F520E866F16
:109B8000490E876F4E0E886F540E896F200E8A6FB4
:109B9000460E8B6F4C0E8C6F410E8D6F530E8E6F79
:109BA000480E8F6F906B560E916F430E926F936FAE
:109BB000200E946F530E956F480E966F4F0E976F51
:109BC000570E986F996B410E9A6F440E9B6F430E20
:109BD0009C6F200E9D6F530E9E6F480E9F6F4F0E11
:109BE000A06F570EA16FA26B540EA36F450EA46F0A
:109BF000530EA56F540EA66F200EA76F4C0EA86FC4
:109C0000410EA96F530EAA6F450EAB6F520EAC6F8B
:109C1000530EAD6FAE6B540EAF6F450EB06F530E5B
:109C2000B16F540EB26F200EB36F540EB46F450E69
:109C3000B56F4D0EB66F500EB76FB86B540EB96F4F
:109C4000450EBA6F530EBB6F540EBC6F200EBD6F26
:109C5000420EBE6F410EBF6F540EC06FC16FC26B1C
:109C6000C36F450EC46F530EC56F540EC66F200EE2
:109C7000C76F410EC86F440EC96F430ECA6FCB6BDE
:109C8000450ECC6FCD6F500ECE6F520ECF6F4F0E74
:109C9000D06F4D0ED16FD26B450ED36F580ED46F6F
:109CA000490ED56F540ED66FD76BD08EC26A0F0E89
:109CB000C112000121EF0FF035EF0FF00601DA6B52
:109CC00000013CEC0FF069EC0FF0500E0601D86F6C
:109CD000000178EF0FF07CEC0FF088EF0FF031EF20
:109CE00010F001EF11F023EF11F08DEC11F097EF70
:109CF00011F0316A640E306E090E0601D96F000151
:109D0000A1EC11F0C00EF212040078EF4AF0FCD77B
:029D100003004E
:020000040030CA
:0E00000000250E0F83018100FFC0FFE0FF40CE
:00000001FF
